:020000020000FC
:100000000C94944D18951895189518951895189561
:100010001895189518951895189518951895189578
:100020001895189518951895189518951895189568
:100030001895189518951895189518950C94BD2F26
:1000400018951895189518950C94B5481895189505
:100050001895189518951895189518951895189538
:100060001895189518951895189518951895189528
:1000700018951895189518950C948F4818951895FB
:100080001895189518951895189518950D0A20002B
:100090000D0A0A205B434D2D352056657273696F3A
:1000A0006E20312E31335D000D0A20546F737320A2
:1000B0004D6F64650D0A000D0A202D3E5B44796E7C
:1000C000616D6978656C5D3A000D0A203C2D5B44DA
:1000D000796E616D6978656C5D3A000D0A203C2D82
:1000E0003E50433A00203C2D3E44796E616D697864
:1000F000656C3A000D0A2041726520796F75207396
:10010000757265203F28792F4E29000D0A205573FE
:10011000616765203A20476F205B506F736974698F
:100120006F6E20416E676C6528307830307E307895
:10013000336666295D000D0A20416C6C2044796E9F
:10014000616D6978656C27732049442077696C6C10
:100150002062652073657420746F20002E20417228
:100160006520796F7520737572653F28592F4E2968
:10017000000D0A204572726F72315B436865636BD4
:100180002044796E616D6978656C2056657273697B
:100190006F6E206973206D6F7265207468616E20C8
:1001A000335D000D0A2042284265666F7265292C76
:1001B0004E284E657874292C512851756974290090
:1001C0000D0A203438354D6F6E69746F72205B4CA8
:1001D000462C43522061726520616464656420612D
:1001E000742070617573652074696D655D0D0A001A
:1001F0000D0A204E6F20446174615B61742042726D
:100200006F61646361737420494420307846455DB2
:10021000000D0A204E6F20446174612843686563B5
:100220006B2049442C204F7065726174696E6720A1
:100230004D6F64652C20426175642072617465297C
:1002400000204C454E3A000D0A204C454420426C9B
:10025000696E6B2049443A002044796E616D69787B
:10026000656C7320466F756E642E000D0A204C4538
:100270004420426C696E6B2049443A000D20466F61
:10028000756E642120424155445F5245473A002C27
:100290002049443A000D0A20426175642052656786
:1002A000206973206368616E67656420746F200045
:1002B000425053000D0A2049443A30202D20000DB1
:1002C0000A2044656C61793A000D0A20546F7271FE
:1002D000756520456E61626C65000D0A204D6F7674
:1002E000652030203C2D3E203078336666000D0AB4
:1002F00020416E79204B657920746F20436F6E74B6
:10030000696E75652E2E2E000D0A205B45455052F4
:100310004F4D20415245415D0D0A204D4F44454C03
:100320005F4E554D4245525F4C202020202020201A
:1003300020285229205B000D0A204D4F44454C5F78
:100340004E554D4245525F4820202020202020203D
:10035000285229205B000D0A2056455253494F4E22
:100360002020202020202020202020202020202885
:100370005229205B000D0A20494420202020202003
:100380002020202020202020202020202028522F24
:1003900057295B000D0A20424155445F52415445A4
:1003A00020202020202020202020202028522F57CD
:1003B000295B000D0A2052455455524E5F44454C6E
:1003C00041595F54494D452020202028522F57295C
:1003D0005B000D0A2043575F414E474C455F4C4937
:1003E0004D49545F4C202020202028522F57295B54
:1003F000000D0A2043575F414E474C455F4C494D25
:1004000049545F48202020202028522F57295B0084
:100410000D0A204343575F414E474C455F4C494DC1
:1004200049545F4C2020202028522F57295B000D73
:100430000A204343575F414E474C455F4C494D4965
:10044000545F482020202028522F57295B000D0A96
:10045000202852455345525645442920202020202B
:1004600020202020202028522F57295B000D0A2011
:100470004C494D49545F54454D5045524154555295
:10048000452020202028522F57295B000D0A2044A8
:100490004F574E5F4C494D49545F564F4C5441475E
:1004A0004520202028522F57295B000D0A20555047
:1004B0005F4C494D49545F564F4C544147452020AD
:1004C00020202028522F57295B000D0A204D41582B
:1004D0005F544F525155455F4C2020202020202052
:1004E000202028522F57295B000D0A204D41585FCC
:1004F000544F525155455F48202020202020202075
:100500002028522F57295B000D0A2052455455527E
:100510004E5F4C4556454C20202020202020202096
:1005200028522F57295B000D0A20414C41524D5F44
:100530004C4544202020202020202020202020283E
:10054000522F57295B000D0A20414C41524D5F53F9
:10055000485554444F574E20202020202020285218
:100560002F57295B000D0A20285245534552564506
:100570004429202020202020202020202028522F05
:1005800057295B000D0A20444F574E5F43414C49A9
:1005900042524154494F4E5F4C20202028522F5741
:1005A000295B000D0A20444F574E5F43414C49429E
:1005B000524154494F4E5F4820202028522F57293E
:1005C0005B000D0A2055505F43414C494252415453
:1005D000494F4E5F4C202020202028522F57295B66
:1005E000000D0A2055505F43414C49425241544945
:1005F0004F4E5F48202020202028522F57295B0093
:100600000D0A205B52414D20415245415D0D0A20AB
:10061000544F525155455F454E41424C4520202094
:10062000202020202028522F57295B000D0A204C23
:100630004544202020202020202020202020202071
:100640002020202028522F57295B000D0A204357D5
:100650005F434F4D504C49414E43455F4D415247DA
:10066000494E2028522F57295B000D0A204343573B
:100670005F434F4D504C49414E43455F4D415247BA
:10068000494E28522F57295B000D0A2043575F43DC
:100690004F4D504C49414E43455F534C4F504520C0
:1006A0002028522F57295B000D0A204343575F43F0
:1006B0004F4D504C49414E43455F534C4F504520A0
:1006C00028522F57295B000D0A20474F414C5F509D
:1006D0004F534954494F4E5F4C2020202020202862
:1006E000522F57295B000D0A20474F414C5F504F56
:1006F000534954494F4E5F48202020202020285243
:100700002F57295B000D0A204D4F56494E475F5326
:10071000504545445F4C2020202020202028522F87
:1007200057295B000D0A204D4F56494E475F5350E5
:100730004545445F482020202020202028522F5764
:10074000295B000D0A20544F525155455F4C494DCD
:1007500049545F4C2020202020202028522F572948
:100760005B000D0A20544F525155455F4C494D498D
:10077000545F482020202020202028522F57295B1A
:10078000000D0A2050524553454E545F504F534977
:1007900054494F4E5F4C20202020285229205B00D6
:1007A0000D0A2050524553454E545F504F53495403
:1007B000494F4E5F4820202020285229205B000D01
:1007C0000A2050524553454E545F53504545445FAF
:1007D0004C20202020202020285229205B000D0AB8
:1007E0002050524553454E545F53504545445F4851
:1007F00020202020202020285229205B000D0A20C4
:1008000050524553454E545F4C4F41445F4C20205D
:10081000202020202020285229205B000D0A205073
:10082000524553454E545F4C4F41445F4820202071
:100830002020202020285229205B000D0A20505221
:100840004553454E545F564F4C5441474520202058
:1008500020202020285229205B000D0A20505245DC
:1008600053454E545F54454D5045524154555245A1
:10087000202020285229205B000D0A20524547499C
:100880005354455245445F494E53545255432E20CC
:100890002028522F57295B000D0A205245534552FC
:1008A0005645442850415553455F54494D452920EC
:1008B00028522F57295B000D0A204D4F56494E47AD
:1008C0002020202020202020202020202020202028
:1008D000285229205B000D0A204C4F434B2020203A
:1008E00020202020202020202020202020202852CE
:1008F0002F57295B000D0A2050554E43485F4C206E
:100900002020202020202020202020202028522F9E
:1009100057295B000D0A2050554E43485F48202060
:1009200020202020202020202020202028522F5747
:10093000295B000D0A0A2044554D50284429203ACD
:100940002044756D7020636F6E74726F6C207461DB
:10095000626C652E000D0A204944205B49445F4EBD
:10096000554D5D203A20536574204944206F662020
:1009700064796E616D6978656C2E000D0A204349BB
:1009800044205B49445F4E554D5D203A20436861E9
:100990006E676520436F6E74726F6C2049442E0041
:1009A0000D0A2052454144205B414444525D5B4C5A
:1009B000454E5D203A205265616420646174612E69
:1009C0002065782952656164203130203220285218
:1009D0006561642066726F6D20307831302C206C38
:1009E000656E677468203229000D0A2057524954F9
:1009F00045205B414444525D5B44415441315D2E8E
:100A00002E203A20577269746520646174612E202B
:100A100065782957726974652031342C3120285744
:100A20007269746520312061742030783134290076
:100A30000D0A205245475F5752205B414444525DA6
:100A40005B44415441315D2E2E203A205265676946
:100A50007374657220777269746520696E7374753A
:100A6000726374696F6E000D0A20414354494F4E02
:100A7000203A20416374696F6E205245475F575298
:100A800020696E737472756374696F6E000D0A204D
:100A9000476F205B504F534954494F4E5D5B535055
:100AA0004545445D3A20476F746F20746865207037
:100AB0006F736974696F6E207769746820746865F4
:100AC0002073706565642E000D0A20484558205B30
:100AD0004E554D5D5B4E554D5D2E2E2E203A2054C9
:100AE00072616E736D6974652072617720646174E0
:100AF000612E2065782948657820464620464620A4
:100B00003031203033000D0A205245534554203AED
:100B10002044796E616D6978656C205265736574E7
:100B20002E000D0A2050494E47205B4E554D5D3A30
:100B3000206578292050696E67204E554D20494424
:100B40002064796E616D6978656C2E000D0A205302
:100B50005752205B414444525D5B4C454E5D5B49BE
:100B6000445D5B444154415D2E2E2E5B49445D5BE8
:100B7000444154415D2E2E2E203A2053796E63203D
:100B800057726974652E000D0A205343414E205B55
:100B90004E554D5D203A205343414E206C696E6B9B
:100BA00065642064796E616D6978656C20696E207A
:100BB000307E4E554D20696E2063757272656E747D
:100BC000206261756420726174652E000D0A204CEC
:100BD0004544205B4E554D5D203A20426C696E6B5A
:100BE000204C4544206F66204E554D2049442E2010
:100BF0002742272C274E2720666F72204944206306
:100C000068616E67652E2027512720666F7220511C
:100C10007569742E000D0A2042415544205B4E55E3
:100C20004D5D203A205365742062617564207261C5
:100C300074652020657829204241554420323228AD
:100C40003537363030425053292C2042415544200C
:100C50003128314D42505329000D0A20534541524D
:100C60004348203A205365617263682049442061FB
:100C70006E64206261756472617465206F662061C4
:100C80006C6C206C696E6B65642064796E616D6953
:100C900078656C732E000D0A2055706461746520B0
:100CA0005B53544152545F49445D205B454E445F61
:100CB00049445D203A2044796E616D6978656C2005
:100CC0006669726D77617265207570646174652EF6
:100CD0002873797374656D2075736572206F6E6CFF
:100CE0007929000D0A0A2020202020202020436F8F
:100CF0007079726967687420524F424F544953208B
:100D0000434F2E2C4C54442E0D0A005B496E7661E5
:100D10006C6964205061676520526561643A000D1A
:100D20000A205B4572723A5278442054696D656FAF
:100D300075745D000D0A205B4572723A57726F6ED2
:100D400067204865616465725D000D0A205B45722D
:100D5000723A5478494420213D20527849445D003C
:100D60000D0A205B4572723A57726F6E67204C65B0
:100D70006E6774685D000D0A205B4572723A5772A7
:100D80006F6E6720436865636B53756D5D000D0A78
:100D900020555044415445205B53544152542049FE
:100DA000445D205B454E442049445D005D3A000DA2
:100DB0000A2049443A00205374616E6462792E001F
:100DC0002057726974696E672E2E00205375636315
:100DD0006573732E00204572726F722E000D0A200B
:100DE0004572722049443A002042616420436F6D8D
:100DF0006D616E64005B457869745D005B53544FB0
:100E0000505D000D0A204D4F54494F4E20504C412B
:100E10005920504147452020202028522F57290093
:100E20000D0A204F4E20504C4159494E47204D4FFE
:100E300054494F4E2020202028522920000D0A20FE
:100E4000545820574952454C455353205041434B29
:100E50004554202028522F5729000D0A205258208F
:100E6000574952454C455353205041434B4554201C
:100E7000202028522920000D0A204E45572050419D
:100E8000434B455420415252495645442020202886
:100E9000522920000D0A20415558204C454420205D
:100EA000202020202020202020202028522F5729B9
:100EB000000D0A20425554544F4E282D532D552DC8
:100EC000442D4C2D522920202028522920000D0A83
:100ED0002054494D4552283132356D5365632045C4
:100EE000616368292028522F5729000D0A205A498A
:100EF0004742454520494420202020202020202012
:100F0000202028522F5729000D0A20524F424F54BB
:100F1000204944202020202020202020202020287C
:100F2000522F5729000D44796E616D6978656C20E8
:100F300020302830783030295B202020205D000DC3
:100F40000A44796E616D6978656C202031283078AB
:100F50003031295B202020205D0020506167654EE4
:100F6000756D6265723A000D0A44796E616D69783B
:100F7000656C2020322830783032295B20202020F8
:100F80005D0020416464723A000D0A44796E616D1F
:100F90006978656C2020332830783033295B202035
:100FA00020205D00202852657365727665642920D3
:100FB0003A000D0A44796E616D6978656C202034C1
:100FC0002830783034295B202020205D002020202C
:100FD000506C6179436F756E743A000D0A44796EF6
:100FE000616D6978656C2020352830783035295B53
:100FF000202020205D00202852657365727665648C
:1010000029203A000D0A44796E616D6978656C207B
:1010100020362830783036295B202020205D0020C3
:1010200028526573657276656429203A000D0A447A
:10103000796E616D6978656C20203728307830379B
:10104000295B202020205D00202852657365727680
:10105000656429203A000D0A44796E616D697865EE
:101060006C2020382830783038295B202020205D03
:10107000002028526573657276656429203A000D58
:101080000A44796E616D6978656C20203928307862
:101090003039295B202020205D002020205061670E
:1010A0006520537465703A000D0A44796E616D696C
:1010B00078656C2031302830783041295B20202041
:1010C000205D0020436F6E74726F6C436F64653AED
:1010D000000D0A44796E616D6978656C20313128A4
:1010E00030783042295B202020205D002020506194
:1010F00067652053706565643A000D0A44796E6136
:101100006D6978656C2031322830783043295B2056
:101110002020205D0020202044584C205365747509
:10112000703A000D0A44796E616D6978656C203102
:10113000332830783044295B202020205D00202097
:10114000416363656C2054696D653A000D0A44790A
:101150006E616D6978656C203134283078304529AE
:101160005B202020205D004C696E6B20746F204E48
:101170006578743A000D0A44796E616D6978656C22
:101180002031352830783046295B202020205D0032
:101190004C696E6B20746F20457869743A000D0AB3
:1011A00044796E616D6978656C203136283078310C
:1011B00030295B202020205D0028526573657276FF
:1011C00065645031293A000D0A44796E616D697881
:1011D000656C2031372830783131295B2020202080
:1011E0005D002852657365727665645231293A0054
:1011F0000D0A44796E616D6978656C20313828304C
:10120000783132295B202020205D002852657365EB
:10121000727665645032293A000D0A44796E616D28
:101220006978656C2031392830783133295B20208A
:1012300020205D00285265736572766564523229FC
:101240003A000D0A44796E616D6978656C20323020
:101250002830783134295B202020205D000D0A449D
:10126000796E616D6978656C20323128307831355E
:10127000295B202020205D000D0A44796E616D6994
:1012800078656C2032322830783136295B20202076
:10129000205D000D0A44796E616D6978656C2032BD
:1012A000332830783137295B202020205D000D0A5B
:1012B00044796E616D6978656C20323428307831FC
:1012C00038295B202020205D000D0A44796E616D75
:1012D0006978656C2032352830783139295B2020D7
:1012E00020205D000D0A44796E616D6978656C207F
:1012F00032362830783161295B202020205D000DB6
:101300000A44796E616D6978656C203237283078CF
:101310003162295B202020205D000D0A44796E6136
:101320006D6978656C2032382830783163295B200C
:101330002020205D000D0A44796E616D6978656C2E
:101340002032392830783164295B202020205D004C
:101350000D0A44796E616D6978656C2033302830F0
:10136000783165295B202020205D000D0A20202097
:10137000506175736554696D652020202020202000
:101380005B2020205D000D0A2020205370656564DD
:1013900020202020202020202020205B2020205DD5
:1013A000202020202020202020202020202020203D
:1013B000202020202020202020202020202020202D
:1013C000202020205B583A2D2D2C593A2D2D2C41D0
:1013D0003A2D2D2D2D5D000D0A20202020202020CB
:1013E000202020202020202020202020535450374F
:1013F00020205354503020535450312053545032F5
:1014000020535450332053545034205354503520DB
:101410005354503620202020476F20537465703A73
:101420002020202020000D0A202020202020202005
:1014300020202020202020202020202020202020AC
:10144000204D53545220534C4156204F4653542064
:10145000202020202020202020202020202020208C
:1014600020202020202020476F20537465703A20D0
:1014700020202020000D0A5D205F20202020202039
:10148000202020202020202020202020202020205C
:10149000202020202020202020202020202020204C
:1014A000202020202020202020202020202020203C
:1014B000202020202020202020202020202020202C
:1014C000202020002041726520796F75207375728D
:1014D000653F5B792F4E5D0020496E76616C6964D3
:1014E00020506167650020496E76616C6964205008
:1014F0006172616D6574657200204F666673657414
:10150000205570646174656400204F7574206F66A7
:101510002052616E676500204F4B000D0A2020208D
:1015200020202020202D434D3A2052503D2850614C
:101530007261302C4F502C506172613129204C4B1C
:10154000205253205B414444525D2020000D0A206C
:10155000427265616B20617420000D0A2045525271
:101560004F523A004946202020202000454C534548
:1015700020494600454C534520202000616E642FD1
:101580006F7220004A554D50202020004C4F41449E
:1015900020202000434F4D50555445005354415294
:1015A00054202000454E44202020200043414C4C34
:1015B0002020200052455455524E20004E554C4C90
:1015C000202020000D0A204845584120444953500E
:1015D0004C4159204D4F4445000D0A204445434994
:1015E0004D414C20444953504C4159204D4F4445A6
:1015F0000003404C464D4840454A230102030A225D
:101600002121217D7D7D7D7D7D7D7D7D7D7D7D7D1E
:101610007D7D797673716E6C6967656361605E5C10
:101620005B59585755545351504F4E4D4C4B4A49A6
:10163000484746454443424241403F3F3E3D3C3C93
:101640003B3A39393837373636353434333332313B
:101650003130302F2F2E2D2D2C2C2B2B2A2A2929BF
:10166000282827272626252525242423232222212E
:10167000212020201F1F1E1E1D1D1D1C1C1B1B1A90
:101680001A1A1919181818171716161615151414EA
:1016900014131312121211111010100F0F0E0E0E40
:1016A0000D0D0C0C0C0B0B0A0A0909090808070799
:1016B00007060605050404040303020201010100F4
:1016C000000000000000000000000000000000001A
:1016D000000000000000000000000000000000000A
:1016E00000000000000000000000000000000000FA
:1016F00000000000000000000000000000000000EA
:1017000000000000000001010102000200010101CF
:1017100001020001010101020002000101010101B9
:1017200001020002000200020002000200010101A9
:10173000010101020001010200020000000001019C
:10174000010101000001010101010001010101018C
:101750000100000101000000000000010000000184
:10176000010200010100000101010102000200016B
:011770000177
:10177200682FA901812F0023B9F40FE003BF00E015
:1017820002BF09E01DE30E94EC4D10E0003021E0B1
:10179200120710F000E009C001BF082F00FB07B7D5
:1017A20001F907BF01E001C000E0862F089500E0C3
:1017B2000093610002B901BB04BB07BB0ABB00E096
:1017C200009365000093620003B902BB05BB08BB2E
:1017D20000B50B7F00BD00B50B7F00BD00E000939C
:1017E200610002B901BB04BB07BB0ABB00E0009366
:1017F20065000093620003B902BB05BB08BBBD9A3A
:10180200C59A909A1C9A1D9A1E9A1F9A04B30F6742
:1018120004BB02B10C6002B9AC9AAB9AAA9AA99A1B
:10182200A89AAE9AAD9AAC9AAB9AAA9AA99AA89A91
:101832001A981B9A01B3006701BB9798949A959ADC
:101842009698AC9AAB9AAA9AA99AA89A0895002354
:1018520091F400E00093900019B902E00BB908E19D
:101862000AB920FB0EF4579A06E0009395000FEF99
:101872000CB95E9A08950130E9F400E000939800F3
:101882001093990002E000939B0008E100939A00F4
:1018920020FB2EF400919A00006800939A0006E063
:1018A20000939D000FEF00939C0000919B00006449
:1018B20000939B000895592F482F80E090E008C0C4
:1018C2002FE93FE021503040E9F700C000000196C7
:1018D20080179107A8F3842F952F08959A938A93DE
:1018E20080E090E098D20A3318F00753102F02C01C
:1018F2000053102F012F10E0102F00E0110F110FD5
:10190200110F110F802B912B86D20A3318F0075337
:10191200102F02C00053102F012F302F20E0822BF6
:10192200932B79D20A3318F00753102F02C00053B9
:10193200102F012F10E044E00E94E04D802B912BEC
:101942006AD20A3318F00753102F02C00053102F27
:10195200012F10E0802B912B8C0189919991089590
:101962000E94824E24972A833B83B02FD12E7A0184
:1019720082E090E001E00093E80CBB249699B394D6
:10198200CC249599C394969A959825C0949801E091
:1019920010E091DF00E00093FE0C0093FD0C949A9E
:1019A20005E010E088DF01E205D101E311E083DF09
:1019B20008E000D10091FD0C1091FE0C011751F0CE
:1019C2000091FD0C1091FE0C011721F024D201327E
:1019D200B9F791E08A95813010F09923B9F29923F1
:1019E20009F4B1C000E00093FE0C0093FD0C442406
:1019F200552466247724A0E08824992409E6DAD0C5
:101A020008E0D8D008D20A33E9F705D2088303D216
:101A1200098301D20A33E9F761DF2801FCD10A33D5
:101A2200E9F75CDF38010881003319F409810634D3
:101A320031F002E6BFD000E3BDD006E6BBD00FEF27
:101A420060160FEF700649F0E6D10A33E9F7E3D1E9
:101A5200093511F4A1E001C0A0E00EE110E02BDF96
:101A620000E00093FE0C0093FD0C02E5A3D008E019
:101A7200A1D0D1D1802F8C3641F4CDD10A33E9F7F0
:101A82002DDF4801AA24A39403C08F3691F7AA241C
:101A9200E2EEFCE040825182E4EEFCE06082718280
:101AA200E6EEFCE080829182B0FBC6F404E110E035
:101AB20002DF04E47FD008E07DD0ADD10A33E9F73C
:101AC20005E010E0F8DE0A811B817BD108E072D0CC
:101AD20008E070D008E06ED008E06CD0B1FB4EF4A4
:101AE20004E110E0E8DEDA1621F007E563D008E051
:101AF20061D0B2FBCEF4AA20B9F004E110E0DBDE43
:101B020003E458D008E056D086D10A33E9F705E05D
:101B120010E0D1DE870155D108E04CD008E04AD070
:101B220008E048D008E046D004E110E0C4DE05E455
:101B320041D008E03FD0949801E010E0BCDE949AD6
:101B420004E610E0B8DE00E00093FE0C0093FD0C0A
:101B52000B2D00FD969A00FF96980C2D00FD959A8C
:101B620000FF959800E00093E80C092F2496E0E12D
:101B72000C94934E5E9A1B981A9A18D05E9BFECFD5
:101B82001A981B9A08958A93802F082F02950F7036
:101B9200005D0A3308F0095F0DD08F70805D082F59
:101BA2000A3308F0095F06D0899108955D9BFECF44
:101BB2000CB90895A99810919B00212F25FFFBCF06
:101BC20000939C0008959A938A93802F082F44E6ED
:101BD2000E94C24D902F092F005DECDF04E6909F1A
:101BE2008019082F4AE00E94C24D902F092F005DF4
:101BF200E1DF0AE0909F8019805D082FDBDF899189
:101C0200999108950E94844E48015901DD24BB2018
:101C120052F49094A094B094000B8194900AA00A7C
:101C2200B00A0DE2C7DF80E09AECAAE9BBE3CC245C
:101C32001AC0DD2019F08201005DBCDF8201930130
:101C4200AC01BD010E94114E801A910AA20AB30A88
:101C52008C019D014AE050E060E070E00E945B4E22
:101C6200C801D901C39409E0C016A8F48401950102
:101C7200AC01BD010E945B4E402E552466247724A0
:101C8200042D052906290729A1F28201005D92DFB0
:101C9200DD24D394D3CF84019501AC01BD010E9410
:101CA2005B4E402E552466247724042D005D82DF8E
:101CB200EEE00C94954E0E948A4E38015524A0E124
:101CC200B7E244240FC000E375DF8C01AD010E942E
:101CD200D04D601A710A8D014AE050E00E94EC4D2D
:101CE200D801439405E04016D0F48301AD010E946F
:101CF200EC4DC801082F092B31F0082F005D5ADF87
:101D020055245394E2CF552021F0082F005D52DF75
:101D1200DCCF04E04016B8F600E24CDFD6CFE8E0B4
:101D22000C949B4E10915F09112311F02CDF089542
:101D320023E010E00AD0089520915F09222311F0D8
:101D420040D0089524E001D008950E94884E3801C1
:101D5200822E5524A0E1B7E244240FC000E32ADF1B
:101D62008C01AD010E94D04D601A710A8D014AE0CA
:101D720050E00E94EC4DD801439405E04016F0F487
:101D82008301AD010E94EC4DC80104E010E0242D56
:101D920030E0021B130B9924081519050CF7082FC4
:101DA200092B31F0082F005D05DF55245394D8CF5D
:101DB2005520A1F2082F005DFDDED2CFEAE00C949F
:101DC200994E9A938A93C8018C01012F10E0DBDEB1
:101DD200082FD9DE8991999108950E948E4EC801EB
:101DE200D9018C019D01022F132F330F220B330BCC
:101DF200E8DF8C01E6DFE4E00C949F4EBA93AA93ED
:101E0200D80103C00C91D6DE11960C910023D1F7B4
:101E1200A991B99108950091FE0C1091FD0C011742
:101E2200D1F30091FE0C102F13951093FE0C10E0CD
:101E32000F701070F801E150F34F008108958A93FA
:101E4200802F082FC0DE08E2B5DE00E3B3DE08E52E
:101E5200B1DE082F98DE09E2ADDE899108950E9475
:101E6200874EEF97EF97EF972797A898992401E06D
:101E72000093680901E00093670905C004E110E0DE
:101E82001ADD08E001BD992011F00C94081806EA49
:101E920015E0B4DF00915809D2DF0FEA15E0AEDF9A
:101EA20020E08E0108571F4F0E94B91F00E00883EF
:101EB200AE0148575F4F9E01205F3F4F8E010E9447
:101EC2000D1E802E00916509009366098820D9F2C3
:101ED2000FE1801610F00EE1802E2AE536E08E0129
:101EE2000E94EB1D002351F628E536E08E010E9488
:101EF200EB1D002309F450C007EB10E00E94C04B19
:101F020080E01CC0FE017096082F10E0000F111F28
:101F1200000F111FE00FF11F008111812281338117
:101F220090E0FC01E553F74F008390E0FC01E5539C
:101F3200F74F0081F7DE00E23DDE839590E0E82D69
:101F4200F0E031978E179F07ECF21B981A9A80E007
:101F520008C090E0FC01E553F74F008127DE5E9A4E
:101F6200839590E0E82DF0E031978E179F078CF370
:101F72005E9BFECF1A981B9A0FEF0E946549009351
:101F8200690909EC10E00E94C04B2091690907E140
:101F920018E00E94724A77CF23E536E08E010E9454
:101FA200EB1D002371F420E536E08E010E94EB1D4B
:101FB200002339F42EE436E08E010E94EB1D00234B
:101FC20069F100915809083CB1F40CE810E00E9454
:101FD200C04B088919892A893B8931DF0AE3EADD86
:101FE200088919892A893B89102F009158090E9472
:101FF200583CA2DE48CF088919892A893B89009377
:1020020095070C891D892E893F890093960722E046
:1020120012E0009158090E949C4A35CF21EA35E02E
:102022008E010E94EB1D0023A9F014E300915809D0
:102032000E94694DC801282F14E1009158090E949D
:10204200851D892F90E0282F15E1009158090E94E3
:10205200851D19CF2CE935E08E010E94EB1D00236E
:1020620031F114E3009158090E94694DD80114E13D
:10207200009158090E94694DC80116E10091580962
:102082000E94694D080F191F169507950A1B1B0B15
:10209200212F27FF04C00195006810E001C010E065
:1020A200202F1AE0009158090E94851DECCE28E9E4
:1020B20035E08E010E94EB1D002341F001E0009308
:1020C2005F0904EC15E10E94C04BDDCE24E935E046
:1020D2008E010E94EB1D002341F000E000935F0996
:1020E20009ED15E10E94C04BCECE2FE835E08E01FE
:1020F2000E94EB1D0023A9F014E3009158090E94ED
:10210200694DC801282F16E1009158090E94851DCA
:10211200892F90E0282F17E1009158090E94851D10
:10212200B2CE2BE835E08E010E94EB1D002339F47C
:1021320023E835E08E010E94EB1D0023F9F080E0D8
:1021420014C0FE017096082F10E0000F111F000F3F
:10215200111FE00FF11F008111812281338190E074
:10216200FC01EB56F84F00838395881550F38A944F
:10217200282D13E80EEF0E949C4A85CE2DE735E00C
:102182008E010E94EB1D002371F42AE735E08E01D7
:102192000E94EB1D002339F428E735E08E010E94EE
:1021A200EB1D0023A1F100915809083C81F40C8930
:1021B2001D892E893F899801488959896A897B89B5
:1021C2008A01102F009158090E94453B5CCE80E0A5
:1021D20014C0FE017096082F10E0000F111F000FAF
:1021E200111FE00FF11F008111812281338190E0E4
:1021F200FC01EB56F84F00838395881550F38A94BF
:10220200282D13E0009158090E949C4A3CCE21E7F8
:1022120035E08E010E94EB1D002301F180E014C025
:10222200FE017096082F10E0000F111F000F111F02
:10223200E00FF11F008111812281338190E0FC01C6
:10224200EB56F84F00838395881550F38A94282D16
:1022520014E0009158090E949C4A15CE2AE635E006
:102262008E010E94EB1D002339F426E635E08E0133
:102272000E94EB1D0023F9F080E014C0FE0170966D
:10228200082F10E0000F111F000F111FE00FF11FA8
:10229200008111812281338190E0FC01EB56F84FDD
:1022A20000838395881550F38A94282D15E00EEF4C
:1022B2000E949C4AE8CD2FE535E08E010E94EB1D7D
:1022C200002381F00C891D892E893F89202F48899E
:1022D20059896A897B898A01102F009158090E94C5
:1022E200851DD1CD29E535E08E010E94EB1D00232D
:1022F20021F104EF10E00E94C04B8DDD093719F087
:10230200093509F0C0CD01E0801619F40091580991
:1023120004C0088919892A893B8920E016E00E94B5
:102322009C4A002309F4AFCD01E00093580921E053
:1023320030E0A9010E94BE4DA6CD22E535E08E0116
:102342000E94EB1D0023A1F001E0801639F420E089
:1023520017E0009158090E949C4A95CD20E017E0B1
:10236200488959896A897B89042F0E949C4A8BCDAE
:102372002FE435E08E010E94EB1D002339F42DE499
:1023820035E08E010E94EB1D0023D9F102E0801698
:1023920019F003E0801681F50EE100939507088994
:1023A20019892A893B8900939607088919892A89FC
:1023B2003B89012F10E00093970703E08016A9F4F0
:1023C2000C891D892E893F89009398070C891D89E4
:1023D2002E893F89012F10E00093990725E013E031
:1023E200009158090E949C4A4ECD23E013E00091CF
:1023F20058090E949C4A47CD0BE011E00E94C04B55
:1024020042CD28E435E08E010E94EB1D002379F0D5
:1024120001E0801619F40091580904C0088919894D
:102422002A893B8920E011E00E949C4A2CCD25E4B8
:1024320035E08E010E94EB1D002349F103E0009379
:102442009507088919892A893B890093960706E32B
:1024520011E00E94C04B0091960764DC0CE511E08C
:102462000E94C04BD8DC093519F0093709F00BCDB1
:1024720022E013E00EEF0E949C4A0091960700931F
:10248200580921E030E0A9010E94BE4DFCCC20E4B5
:1024920035E08E010E94EB1D002339F42BE036E07B
:1024A2008E010E94EB1D0023E1F000915809083CC7
:1024B20011F400D6E8CC00E0009395070AE30093FC
:1024C200960722E012E0009158090E949C4A0023DC
:1024D20009F4D9CC009158090E3F09F4D4CCEAD5BD
:1024E200D2CC24E036E08E010E94EB1D002309F4D9
:1024F200A5C103E0801651F4488859886A887B8810
:102502000C891D892E893F89A02E0DC002E08016FC
:1025120031F4488859886A887B88A42C04C00EE864
:102522001DE00E94C04B02E0801621F003E08016FD
:1025320009F0A9CC00E0009367090093680909B18A
:10254200023289F421E014E00EEF0E947F4D0AE08E
:1025520010E0B1D901E009B90093570920E030E059
:10256200A9010E94BE4D22E214E00EEF0E947F4DAF
:102572000AE010E0A0D902E209B90093570920E06D
:1025820030E0A9010E94BE4D21E014E00EEF0E944E
:102592007F4D0AE010E08FD901E009B90093570995
:1025A20020E030E0A9010E94BE4D00E00E94DB4B1A
:1025B20005C001E711E00E94C04B4394A41408F443
:1025C2001EC15524F201E659F64F00810023A9F3FA
:1025D20009B1013049F001E009B90093570920E03F
:1025E20030E0A9010E94BE4D0FEA1DE00E94C04BDF
:1025F200042D98DB90E0992399F491E080E08F31EB
:10260200D0F7082F0E94BD1D002341F020E011E009
:10261200082F0E949C4A002309F490E08395EFCF93
:1026220006EB1DE00E94C04B80E00FC0841561F0F4
:1026320090E0FC01E659F64F0081002329F025E0E5
:102642001DE2082F0E94851D83958F3178F300ECDF
:102652001DE00E94C04B2FEF1AEF042D0E94851D32
:102662002EEF1DE2042D0E94851D002309F4A1CF47
:1026720003E0502E02E209B90093570920E030E04E
:10268200A9010E94BE4D04E610E015D90DE072DAF0
:1026920000E00E943F1D0CE46DDA00E00E943F1D45
:1026A2001B981A9A80E090ECA0E0B0E0882466249F
:1026B200772412C0FC013A2F3BBF069000E00BBF0B
:1026C2008F5F9F4FAF4FBF4F800C002D6FDA5E9A26
:1026D20001E0600E00E0701E0FEF601607E1700669
:1026E20048F3082D63DA5E9A5E9BFECF1A981B9A16
:1026F20000E00E943F1D06E53DDA00E00E943F1D1A
:1027020000E001C00395043638F410E0F801E95EF8
:10271200F74F10811D32B1F70395202F01C00395A9
:10272200043638F410E0F801E95EF74F10811D32EB
:10273200B1F7039510E001C01395183090F4602FA3
:10274200062F0395422F242F239570E0FB01E95EAB
:10275200F74F308150E0FA01E95EF74F40813417BC
:1027620059F3183031F50BEC1DE00E94C04B01E427
:1027720001DA00E00E943F1D07E4FCD900E00E945C
:102782003F1D04E610E097D801E009B9009357090C
:1027920020E030E0A9010E94BE4D20E017E0042DA8
:1027A2000E949C4A0CE211E086D800E0009367097F
:1027B20004CF05ED1DE00E94C04B5A9409F063CF8F
:1027C20001E4D8D900E00E943F1D07E4D3D900E01C
:1027D2000E943F1D04E610E06ED801E009B90093A3
:1027E200570920E030E0A9010E94BE4D20E017E029
:1027F200042D0E949C4A0CE211E05DD8DECE21E05D
:1028020014E00EEF0E947F4D0AE010E054D801E080
:1028120009B90093570920E030E0A9010E94BE4D9A
:102822000E94894B09B10093570920E030E0A901C9
:102832000E94BE4D01E00093680925CB2FEF35E0E1
:102842008E010E94EB1D002309F440C0B09167097C
:1028520000E0009368090093670980E001E08016B8
:1028620011F4AEEF05C0088919892A893B89A02F86
:102872000CE810E00E94C04B90E005C00DE29AD92E
:102882000DE598D993959A1788F40BE593D9092FFA
:1028920049DA0AE38FD920E011E0092F0E949C4A0D
:1028A200002361F30FE486D98395EACF0CE810E0A8
:1028B2000E94C04B082FC3DA08E512E00E94C04B09
:1028C200B093670901E000936809DDCA2BEF35E098
:1028D2008E010E94EB1D002309F450C001E0801616
:1028E20019F4A091580905C0088919892A893B89D8
:1028F200A02F01E00093670900E00093680903EA52
:1029020011E00E94C04B80E007E412E00E94C04B3D
:102912000A2F08DA0091FE0C1091FD0C011791F0BC
:102922007ADA802F823411F0823609F4AA958E3435
:1029320011F08E3609F4A3950BE612E00E94C04B0B
:102942000A2FF0D921E019E10A2F0E947F4D04E6F7
:1029520010E00E945C0C20E019E10A2F0E947F4DDA
:1029620004E610E00E945C0C813521F0813711F001
:102972008B3181F601E00093680985CA24EF35E0C6
:102982008E010E94EB1D002309F48EC000E000932B
:1029920068090AE00FD980E001C083958E3F08F0F4
:1029A20078C089B920E011E00EEF0E949C4A0DE048
:1029B20001D980FB1EF40BE2FDD802C00AE2FAD86C
:1029C20000916909002309F45DC0A0E056C0B0E09F
:1029D200FD01E95EF74F00810F3F09F04DC00A2F5C
:1029E20010E00F5F1F4FF801E95EF74F00810F3FC4
:1029F20009F042C00A2F10E00D5F1F4FF801E95E97
:102A0200F74F00810230C1F50A2F10E00E5F1F4F11
:102A1200F801E95EF74F408150E00A2F10E00D5FA8
:102A22001F4FF801E95EF74F208130E0240F351F78
:102A32000A2F10E00B5F1F4FF801E95EF74F00818C
:102A420010E0020F131F0F3F20E01207A9F40CE75A
:102A520012E00E94C04B082F65D90FE812E00E94D5
:102A6200C04B0A2F10E00E5F1F4FF801E95EF74FCF
:102A7200008158D90AE09ED8A39500916909A01750
:102A820008F4A5CF0091FE0C1091FD0C011709F47A
:102A920084CF0091570909B901E0009368090DE05C
:102AA20089D800E287D8EFC92FEE35E08E010E9467
:102AB200EB1D002391F104E0009395070889198921
:102AC2002A893B890093960722E013E00EEF0E94C9
:102AD2009C4A05E912E00E94C04B00E814E82EE18E
:102AE20030E0488959896A897B894F5F5F4F6F4F10
:102AF2007F4F0E94354E86D800EB12E00E94C04BF9
:102B0200088919892A893B8909B90093570920E064
:102B120030E0A9010E94BE4DB6C927EE35E08E0114
:102B22000E94EB1D002309F442C001E0801631F43B
:102B320000E1402E55246624772404C04888598831
:102B42006A887B8800EC11E00E94C04B2BC0009188
:102B52006609109165090117A1F080E090E0A0E0FC
:102B6200B0E0AA240091660910E0F801EB56F94F93
:102B72000081E6E6F9E0108113951083D3D800E2D4
:102B820019D88F5F9F4FAF4FBF4F84159505A6058C
:102B9200B705E8F2AA2031F40DE00CD80AE00AD811
:102BA200AA24A39480E090E0A0E0B0E0EECF22EE71
:102BB20035E08E010E94EB1D002309F44AC04888CB
:102BC20059886A887B888C899D89AE89BF8904EB84
:102BD20012E00E94C04B042DA5D80FEB12E00E9418
:102BE200C04B8C01A9D809EC12E00E94C04BA0E0B6
:102BF20006C021E018E10A2F0E947F4DA3954A16D4
:102C0200C0F70AED12E00E94C04B0CC02FEF33E078
:102C12001EE10A2F0E94874DA3954A16B8F78C0130
:102C22000E945C0C0091FE0C1091FD0C011709F042
:102C32002AC9A0E007C020E030E01EE10A2F0E946E
:102C4200874DA3954A16B8F78C010E945C0CA0E050
:102C5200E4CF2EED35E08E01BDD7002309F434C157
:102C620000E000936809009158090093950721E05C
:102C720015E00EEF0E949C4A01E0801641F520E12A
:102C820030E0A9010E94B24D802E80E090E0E82D54
:102C9200F0E031978E179F070CF042C0E82FF0E06A
:102CA2007196AF010E94B24D10E020E030E0FE01CB
:102CB2007096482F50E0440F551F440F551FE40FE4
:102CC200F51F00831183228333838395DFCF05E1D0
:102CD200801610F004E1802E20E130E0082DA901D9
:102CE2000E94BE4D80E015C0FE017096082F10E0D4
:102CF200000F111F000F111FE00FF11F0081118142
:102D020022813381E82FF0E07196AF010E94BE4D1F
:102D1200839590E0E82DF0E031978E179F0724F31A
:102D22000CE810E00E94C04B0BE50E94DB0D80E036
:102D320004C00DE50E94DB0D839590E0E82DF0E0E4
:102D420031978E179F07DCF4FE017096082F10E072
:102D5200000F111F000F111FE00FF11F00811181E1
:102D6200228133810E94930E90E0E82DF0E03297A9
:102D72008E179F07F4F60DE20E94DB0DDDCF009166
:102D8200FE0C1091FD0C011709F099C00CE810E03F
:102D92000E94C04B80E019C0FE017096082F10E01F
:102DA200000F111F000F111FE00FF11F0081118191
:102DB20022813381102F009158090E945A4D0E949E
:102DC200930E00E20E94DB0D839590E0E82DF0E087
:102DD20031978E179F079CF6FE017096082F10E020
:102DE200000F111F000F111FE00FF11F0081118151
:102DF20022813381083CF9F000915809043688F1A8
:102E0200009158090E3668F50BE317E1FE01709642
:102E1200282F30E0220F331F220F331FE20FF31F40
:102E2200408151816281738150E0040F151FF801C6
:102E320004910230B1F4FE017096082F10E0000FE9
:102E4200111F000F111FE00FF11F0081118122815C
:102E52003381102F009158090E94583C0E949D0E08
:102E6200B0CF03E017E1FE017096282F30E0220F69
:102E7200331F220F331FE20FF31F40815181628102
:102E8200738150E0040F151FF8010491023009F01C
:102E920083CFFE017096082F10E0000F111F000F64
:102EA200111FE00FF11F0081118122813381102F48
:102EB200009158090E94694D0E949D0E82CF01E047
:102EC200009368090C94440F29ED35E08E0182D6F7
:102ED200002389F1488859886A887B888C899D8972
:102EE200AE89BF8900E000936809A0E04A1698F015
:102EF20021E018E10A2F0E947F4DA395F7CF2FEF13
:102F020033E01EE10A2F0E94874DA3954A16B8F7B7
:102F12008C010E945C0CA0E007C020E030E01EE1C2
:102F22000A2F0E94874DA3954A16B8F78C010E947A
:102F32005C0CA0E0EBCF25ED35E08E014BD60023F3
:102F420069F0088919892A893B890093580921E087
:102F520030E0A9010E94BE4D0C94440F20ED35E0F3
:102F62008E0138D6002331F42EEC35E08E0132D6B4
:102F7200002321F00E94D6480C94440F28EC35E03F
:102F82008E0128D6002331F426EC35E08E0122D6BC
:102F9200002321F00E9409490C94440F21EC35E0F2
:102FA2008E0118D6002319F03CD00C94440F2DEB5F
:102FB20035E08E010FD6002381F002E0801640F04A
:102FC200088919892A893B890E9413410C94440F6C
:102FD20001E00E9413410C94440F26EB35E08E0170
:102FE200F9D5002331F422EB35E08E01F3D500232D
:102FF20021F0992493940C94440F0CE810E00E9461
:10300200C04B08EE1DE00E94C04B0C94440F00E040
:1030120000936809EF96EF96EF962796EBE00C94F3
:10302200984E03E319E00E94C04B05E519E00E94A7
:10303200C04B0BE719E00E94C04B00EA19E00E9466
:10304200C04B09EE19E00E94C04B00E31AE00E9457
:10305200C04B07E61AE00E94C04B0DE81AE00E943E
:10306200C04B08EC1AE00E94C04B06E01BE00E9435
:10307200C04B02E21BE00E94C04B0CE41BE00E942A
:10308200C04B07E81BE00E94C04B0CEC1BE00E9407
:10309200C04B05E11CE00E94C04B09E51CE00E9408
:1030A200C04B06E91CE00E94C04B03EE1CE00E94EC
:1030B200C04B08950E948E4E00915809083C09F0B9
:1030C200B9C088E103E01EE00E94C04B082F0E94B5
:1030D200200F0AE30E94DB0D182F009158090E946D
:1030E200583C0E949D0E839500E21EE00E94C04B58
:1030F200082F0E94200F0AE30E94DB0D182F009177
:1031020058090E94583C0E949D0E83950DE31EE0D3
:103112000E94C04B082F0E94200F0AE30E94DB0D81
:10312200182F009158090E94583C0E949D0E8395C9
:1031320083950AE51EE00E94C04B082F0E94200FD3
:103142000AE30E94DB0D182F009158090E94583C97
:103152000E949D0E8395839507E71EE00E94C04B57
:10316200082F0E94200F0AE30E94DB0D182F009106
:1031720058090E94583C0E949D0E839504E91EE066
:103182000E94C04B082F0E94200F0AE30E94DB0D11
:10319200182F009158090E94583C0E949D0E839559
:1031A20001EB1EE00E94C04B082F0E94200F0AE391
:1031B2000E94DB0D182F009158090E94583C0E9472
:1031C2009D0E83950EEC1EE00E94C04B082F0E94BC
:1031D200200F0AE30E94DB0D182F009158090E946C
:1031E200583C0E949D0E83950BEE1EE00E94C04B40
:1031F200082F0E94200F0AE30E94DB0D182F009176
:1032020058090E94583C0E949D0E8395839508E0C0
:103212001FE00E94C04B082F0E94200F0AE30E9469
:10322200DB0D182F009158090E94583C0E949D0EF8
:10323200839521C480E008E013E00E94C04B082F70
:103242000E94200F0CEA1DE00E94C04BA82FB0E0A4
:103252001596FD01E95EF74F00810E94200F8395CC
:1032620007E313E00E94C04B082F0E94200F0CEAD4
:103272001DE00E94C04BA82FB0E01596FD01E95E4B
:10328200F74F00810E94200F839506E513E00E940C
:10329200C04B082F0E94200F0CEA1DE00E94C04B79
:1032A200A82FB0E01596FD01E95EF74F00810E945C
:1032B200200F839505E713E00E94C04B082F0E9460
:1032C200200F0CEA1DE00E94C04BA82FB0E015961B
:1032D200FD01E95EF74F00810E94200F839504E90A
:1032E20013E00E94C04B082F0E94200F0CEA1DE041
:1032F2000E94C04BA82FB0E01596FD01E95EF74F82
:1033020000810E94200F839503EB13E00E94C04BC3
:10331200082F0E94200F0CEA1DE00E94C04BA82F2C
:10332200B0E01596FD01E95EF74F00810E94200F83
:10333200839502ED13E00E94C04B082F0E94200FDC
:103342000CEA1DE00E94C04BA82FB0E01596FD01CB
:10335200E95EF74F00810E94200F839501EF13E091
:103362000E94C04B082F0E94200F0CEA1DE00E9411
:10337200C04BA82FB0E01596FD01E95EF74F008122
:103382000E94200F839500E114E00E94C04B082F99
:103392000E94200F0CEA1DE00E94C04BA82FB0E053
:1033A2001596FD01E95EF74F00810E94200F83957B
:1033B2000FE214E00E94C04B082F0E94200F0CEA7B
:1033C2001DE00E94C04BA82FB0E01596FD01E95EFA
:1033D200F74F00810E94200F83950EE414E00E94B3
:1033E200C04B082F0E94200F0CEA1DE00E94C04B28
:1033F200A82FB0E01596FD01E95EF74F00810E940B
:10340200200F83950DE614E00E94C04B082F0E9406
:10341200200F0CEA1DE00E94C04BA82FB0E01596C9
:10342200FD01E95EF74F00810E94200F83950CE8B1
:1034320014E00E94C04B082F0E94200F0CEA1DE0EE
:103442000E94C04BA82FB0E01596FD01E95EF74F30
:1034520000810E94200F83950BEA14E00E94C04B6A
:10346200082F0E94200F0CEA1DE00E94C04BA82FDB
:10347200B0E01596FD01E95EF74F00810E94200F32
:1034820083950AEC14E00E94C04B082F0E94200F83
:103492000CEA1DE00E94C04BA82FB0E01596FD017A
:1034A200E95EF74F00810E94200F839509EE14E038
:1034B2000E94C04B082F0E94200F0CEA1DE00E94C0
:1034C200C04BA82FB0E01596FD01E95EF74F0081D1
:1034D2000E94200F839508E015E00E94C04B082F40
:1034E2000E94200F0CEA1DE00E94C04BA82FB0E002
:1034F2001596FD01E95EF74F00810E94200F83952A
:1035020007E215E00E94C04B082F0E94200F0CEA30
:103512001DE00E94C04BA82FB0E01596FD01E95EA8
:10352200F74F00810E94200F839506E415E00E9468
:10353200C04B082F0E94200F0CEA1DE00E94C04BD6
:10354200A82FB0E01596FD01E95EF74F00810E94B9
:10355200200F839505E615E00E94C04B082F0E94BC
:10356200200F0CEA1DE00E94C04BA82FB0E0159678
:10357200FD01E95EF74F00810E94200F839504E868
:1035820015E00E94C04B082F0E94200F0CEA1DE09C
:103592000E94C04BA82FB0E01596FD01E95EF74FDF
:1035A20000810E94200F839503EA15E00E94C04B20
:1035B200082F0E94200F0CEA1DE00E94C04BA82F8A
:1035C200B0E01596FD01E95EF74F00810E94200FE1
:1035D200839502EC15E00E94C04B082F0E94200F39
:1035E2000CEA1DE00E94C04BA82FB0E01596FD0129
:1035F200E95EF74F00810E94200F839501EE15E0EE
:103602000E94C04B082F0E94200F0CEA1DE00E946E
:10361200C04BA82FB0E01596FD01E95EF74F00817F
:103622000E94200F83950EEE12E00E94C04B0E9472
:103632000C0F00E016E00E94C04B082F0E94200FE2
:103642000CEA1DE00E94C04BA82FB0E01596FD01C8
:10365200E95EF74F00810E94200F83950CE216E08D
:103662000E94C04B082F0E94200F0CEA1DE00E940E
:10367200C04BA82FB0E01596FD01E95EF74F00811F
:103682000E94200F83950BE416E00E94C04B082F86
:103692000E94200F0CEA1DE00E94C04BA82FB0E050
:1036A2001596FD01E95EF74F00810E94200F839578
:1036B2000AE616E00E94C04B082F0E94200F0CEA77
:1036C2001DE00E94C04BA82FB0E01596FD01E95EF7
:1036D200F74F00810E94200F839509E816E00E94AF
:1036E200C04B082F0E94200F0CEA1DE00E94C04B25
:1036F200A82FB0E01596FD01E95EF74F00810E9408
:10370200200F839508EA16E00E94C04B082F0E9402
:10371200200F0CEA1DE00E94C04BA82FB0E01596C6
:10372200FD01E95EF74F00810E94200F839507ECAF
:1037320016E00E94C04B082F0E94200F0CEA1DE0E9
:103742000E94C04BA82FB0E01596FD01E95EF74F2D
:1037520000810E94200F839506EE16E00E94C04B66
:10376200082F0E94200F0CEA1DE00E94C04BA82FD8
:10377200B0E01596FD01E95EF74F00810E94200F2F
:10378200839505E017E00E94C04B082F0E94200F8E
:103792000CEA1DE00E94C04BA82FB0E01596FD0177
:1037A200E95EF74F00810E94200F839504E217E043
:1037B2000E94C04B082F0E94200F0CEA1DE00E94BD
:1037C200C04BA82FB0E01596FD01E95EF74F0081CE
:1037D2000E94200F839503E417E00E94C04B082F3C
:1037E2000E94200F0CEA1DE00E94C04BA82FB0E0FF
:1037F2001596FD01E95EF74F00810E94200F839527
:1038020002E617E00E94C04B082F0E94200F0CEA2C
:103812001DE00E94C04BA82FB0E01596FD01E95EA5
:10382200F74F00810E94200F839501E817E00E9464
:10383200C04B082F0E94200F0CEA1DE00E94C04BD3
:10384200A82FB0E01596FD01E95EF74F00810E94B6
:10385200200F839500EA17E00E94C04B082F0E94B8
:10386200200F0CEA1DE00E94C04BA82FB0E0159675
:10387200FD01E95EF74F00810E94200F83950FEB57
:1038820017E00E94C04B082F0E94200F0CEA1DE097
:103892000E94C04BA82FB0E01596FD01E95EF74FDC
:1038A20000810E94200F83950EED17E00E94C04B0D
:1038B200082F0E94200F0CEA1DE00E94C04BA82F87
:1038C200B0E01596FD01E95EF74F00810E94200FDE
:1038D20083950DEF17E00E94C04B082F0E94200F26
:1038E2000CEA1DE00E94C04BA82FB0E01596FD0126
:1038F200E95EF74F00810E94200F83950CE118E0EA
:103902000E94C04B082F0E94200F0CEA1DE00E946B
:10391200C04BA82FB0E01596FD01E95EF74F00817C
:103922000E94200F83950BE318E00E94C04B082FE2
:103932000E94200F0CEA1DE00E94C04BA82FB0E0AD
:103942001596FD01E95EF74F00810E94200F8395D5
:103952000AE518E00E94C04B082F0E94200F0CEAD3
:103962001DE00E94C04BA82FB0E01596FD01E95E54
:10397200F74F00810E94200F839509E718E00E940B
:10398200C04B082F0E94200F0CEA1DE00E94C04B82
:10399200A82FB0E01596FD01E95EF74F00810E9465
:1039A200200F839508E918E00E94C04B082F0E945F
:1039B200200F0CEA1DE00E94C04BA82FB0E0159624
:1039C200FD01E95EF74F00810E94200F839507EB0E
:1039D20018E00E94C04B082F0E94200F0CEA1DE045
:1039E2000E94C04BA82FB0E01596FD01E95EF74F8B
:1039F20000810E94200F839506ED18E00E94C04BC3
:103A0200082F0E94200F0CEA1DE00E94C04BA82F35
:103A1200B0E01596FD01E95EF74F00810E94200F8C
:103A2200839505EF18E00E94C04B082F0E94200FDB
:103A32000CEA1DE00E94C04BA82FB0E01596FD01D4
:103A4200E95EF74F00810E94200F839504E119E09F
:103A52000E94C04B082F0E94200F0CEA1DE00E941A
:103A6200C04BA82FB0E01596FD01E95EF74F00812B
:103A72000E94200F8395E4E00C949F4E9A938A93C0
:103A8200902F80E000916609109165090117D1F32A
:103A920040E050E060E070E0009166091091650935
:103AA2000117A1F48A019B01A801B9014F5F5F4F81
:103AB2006F4F7F4F013EE3E91E07E4E02E07E0E08F
:103AC2003E0750F3082F8991999108950091660954
:103AD20010E0F801EB56F94F0081E6E6F9E01081BB
:103AE20013951083282F30E0F901E95EF74F008328
:103AF200992341F0082F10E0F801E95EF74F0081A9
:103B02000E94DB0D8395C4CF0E948E4E902FA12F71
:103B1200B22FA0939507B093960700EF00939707F3
:103B220005E5009398070FE0009399070AEA0093CE
:103B32009A0726E01DE0092F0E94214A802F00915A
:103B42006809002349F00CE810E00E94C04B282FBE
:103B52000BEC18E00E94724A0AE010E00E945C0C32
:103B62001A2F092F0E945A4D0B1711F401E001C0C0
:103B720000E0E4E00C949F4E0F3130F410E0F801C5
:103B8200E659F64F00810895043650F00E3640F49F
:103B920010E004561040F801E657F64F00810895F0
:103BA20000E00895A80100E001C00395083C88F4F4
:103BB20010E0F901E00FF11F608110E0FA01E00F5F
:103BC200F11F608310E0F901E00FF11F1081112352
:103BD20061F70895A80100E010E0FA01E00FF11F7B
:103BE200608110E0F901E00FF11F1081611791F47B
:103BF200039510E0FA01E00FF11F1081112339F44F
:103C020010E0F901E00FF11F1081112321F0093CAE
:103C120018F3089500E008950E948B4ED901CA015D
:103C2200442401C043945524FC01E40DF51D208178
:103C32002032C1F32CE3421608F041C05524FC01A6
:103C4200E40DF51D20812223D1F120E021C055246D
:103C5200FC01E40DF51D3081313670F05524FC0174
:103C6200E40DF51D30813B3738F45524FC01E40D99
:103C7200F51D30813F7530835524FC01E40DF51D9F
:103C8200408130E0F801E20FF31F40832395439413
:103C92005524FC01E40DF51D3081303350F05524DC
:103CA200FC01E40DF51D30813B3718F430E1431679
:103CB20070F240E030E0F801E20FF31F4083E02FA2
:103CC200F12F0081002311F400E0A6C066249EC0FB
:103CD20043945524FC01E40DF51D00810032C1F32B
:103CE2005524FC01E40DF51D0081002319F46394B1
:103CF200062D92C000E010E020E030E0462D50E0BA
:103D0200440F551F440F551FFD01E40FF51F00839B
:103D120011832283338342C0062D10E0000F111F4E
:103D2200000F111FFD01E00FF11F0081118122819F
:103D320033814AE050E060E070E00E94114E462D6F
:103D420050E0440F551F440F551FFD01E40FF51FAE
:103D520000831183228333835524FC01E40DF51D76
:103D6200008110E000531040212F220F220B322F2E
:103D7200462D50E0440F551F440F551FFD01E40F1F
:103D8200F51F4081518162817381400F511F621F73
:103D9200731F408351836283738343940CE3401601
:103DA200A0F55524FC01E40DF51D0081002321F44A
:103DB20002E0600E062D30C05524FC01E40DF51D15
:103DC20000810B33E1F05524FC01E40DF51D008167
:103DD2000A33A9F05524FC01E40DF51D00810C32D3
:103DE20071F05524FC01E40DF51D00810E3239F00D
:103DF2005524FC01E40DF51D0081003281F400E23E
:103E02005524FC01E40DF51D008363940EE1601658
:103E120008F45FCF6394062DE7E00C949C4E00916A
:103E22005F09002309F478CF5524FC01E40DF51D48
:103E32000081003308F446C05524FC01E40DF51D51
:103E420000810A33F8F5062D10E0000F111F000F54
:103E5200111FFD01E00FF11F0081118122813381C9
:103E620044E00E942D4E462D50E0440F551F440F52
:103E7200551FFD01E40FF51F008311832283338355
:103E82005524FC01E40DF51D008110E000531040A3
:103E9200212F220F220B322F462D50E0440F551FA7
:103EA200440F551FFD01E40FF51F408151816281CE
:103EB2007381400F511F621F731F408351836283BE
:103EC20073836BCF5524FC01E40DF51D0081013491
:103ED20008F463CF5524FC01E40DF51D00810B3776
:103EE20008F05BCF5524FC01E40DF51D00810F7530
:103EF2000083062D10E0000F111F000F111FFD019E
:103F0200E00FF11F008111812281338144E00E9480
:103F12002D4E462D50E0440F551F440F551FFD01F5
:103F2200E40FF51F00831183228333835524FC01A0
:103F3200E40DF51D008110E007531040212F220FE0
:103F4200220B322F462D50E0440F551F440F551FB0
:103F5200FD01E40FF51F4081518162817381400FA1
:103F6200511F621F731F408351836283738315CF76
:103F72000E948E4EC801A22FB1E016C008E00E9436
:103F8200DB0D00E20E94DB0D08E00E94DB0D0A2F30
:103F9200A02FAA95002391F72EED3DE08C0102DEC1
:103FA200A02F8C010E94FF0EBB23A9F10E940C0FCF
:103FB200102F1050C9F31A9551F3175099F012505F
:103FC20029F0135019F01E5079F319C000E0B0E047
:103FD200FC01EA0FFB1F00839C010EED1DE0E2DDF8
:103FE20001E01AC0A13000F3AA9508E00E94DB0D9F
:103FF20000E20E94DB0D08E00E94DB0DD5CFAC335E
:1040020098F62A2F30E0FC01E20FF31F00830E9492
:10401200DB0DA395C9CF00E0E4E00C949F4E0E9413
:104022008E4E902F812F983050F5883040F5092F11
:1040320010E00F5F1F4F40E450E00E94D04DD801C6
:10404200082F10E00F5F1F4F40E450E00E94D04D58
:1040520020E011C0422F50E0400F511FFA01EB52F5
:10406200F64F3081422F50E04A0F5B1FFA01EB52AC
:10407200F64F30832395203468F3092F03D0E4E010
:104082000C949F4E9A938A93902F973011F490E05C
:1040920001C0939580E007C0182F092F50D2182F26
:1040A200092F2BD183958F31B8F31FE1092F47D206
:1040B2001FE1092FD3D0F801EB52F64F00810E9485
:1040C200930E10E2092F3BD210E2092FC7D0F8015C
:1040D200EB52F64F00810E94930E899199910895B7
:1040E200005049F00A9561F00A9579F00A9591F02D
:1040F2000A95A9F0089504EC14E10E94C04B0895BA
:1041020008ED14E10E94C04B089506EE14E10E94EE
:10411200C04B089509EF14E10E94C04B089509E0D5
:1041220015E10E94C04B08959A938A93802F912F94
:10413200E0E0F6E11491E7EFF5E104910E94852FAA
:1041420022E0082F10E00E94A60EE1E0F6E11491B1
:10415200E8EFF5E104910E94852F22E0092F10E09B
:104162000E94A60EE2E0F6E11491E9EFF5E1049176
:104172000E94852F192F082F71D00E949D0E8991C0
:10418200999108958A93EAEFF5E11491E1EFF5E14F
:1041920004910E94852F80E004C000E20E94DB0DA2
:1041A20083958634D0F3EAEFF5E11491E1EFF5E17E
:1041B20004910E94852F899108959A938A939091F0
:1041C200E90980E00CC0182F00911A0E0395B7D1AF
:1041D20008E00E94DB0D00E20E94DB0D83958F3127
:1041E20090F380E00BC0182F092F0395A8D108E0A7
:1041F2000E94DB0D0CE70E94DB0D83958F3198F353
:1042020090931A0EEEEFF5E11491E5EFF5E10491CA
:104212000E94852F092F0E94930E899199910895EA
:10422200093031F4133020F0143110F401E0089514
:10423200083021F41F3110F401E00895083030F401
:10424200103211F01F3111F401E00895083020F40A
:10425200103210F402E0089500E00895682F202F34
:10426200812F222371F48F3138F4082F10E0000FD0
:10427200111F00501E4F39C0082F10E0015E1D4F64
:1042820034C08F3149F4022F10E040E450E00E9424
:10429200D04D025C1F4F29C0803249F4022F10E03A
:1042A20040E450E00E94D04D015C1F4F1EC02830F8
:1042B20029F4082F10E0005E1F4F17C0293029F49F
:1042C200082F10E0055F1F4F10C0022F10E00150B1
:1042D200104040E450E00E94D04D980102E0809FDF
:1042E2008001020F131F005C1F4F003422E01207EF
:1042F20010F000E010E0862F08959A938A93902F91
:10430200812F8F3108F042C0182F092FA7DFF80143
:10431200EB52F64F20813181203004E0300748F023
:10432200182F092F9BDFF801EB52F64F018107FF8F
:104332000BC0182F092F92DFF801EB52F64F0081C4
:1043420011810E949D0E22C0182F092F87DFF801CC
:10435200EB52F64F018105FF0DC00FE30E94DB0D0A
:104362000FE30E94DB0D0FE30E94DB0D0FE30E94BF
:10437200DB0D0CC00DE20E94DB0D0DE20E94DB0D95
:104382000DE20E94DB0D0DE20E94DB0D89919991F5
:1043920008959A938A930091DA0C002351F000E079
:1043A2009FDE0E940C0F093521F0093711F000E061
:1043B20085C0E8EDFCE00081118120E030E040E0C2
:1043C20052E060E070E00E94114EA801B901405035
:1043D20050426F4F7F4F90E000E010E018C008019C
:1043E20022243324040E151E261E371EF001322D00
:1043F2003BBF069020E02BBFF801EB52F64F008244
:10440200F801EB52F64F2081920F0F5F1F4F0030E1
:1044120022E0120720F380E00DC020E030E402E049
:10442200809F800100501E4FF801EB52F64F20830F
:10443200318383958F3180F5082F10E0F801E6591A
:10444200F64F0081002349F318E1082F0E945A4DCC
:10445200013081F41EE1082F0E94592F22E0829F31
:1044620020E0020E22E0121EF001EB52F64F008312
:104472001183DFCF14E2082F0E94592F00601062CF
:1044820022E0829F20E0020E22E0121EF001EB5297
:10449200F64F00831183CDCF9F3F21F40091E909AC
:1044A200083008F00ED000E00093DA0C0091EC091D
:1044B200053018F000E00093EC0901E08991999130
:1044C20008953B2F2A2FE0E0F0E006C000E0DF0174
:1044D200AB52B64F0C933196E03200E0F007B0F3E6
:1044E200E0E2F0E006C005E5DF01AB52B64F0C9307
:1044F2003196E03400E0F007B0F3E0E4F0E009C008
:1045020000E010E4DF01AB52B64F0D931C931197FC
:104512003296E03002E0F00798F300E00093E909F8
:1045220001E00093E40900E20093EB0900E200934A
:10453200ED0900E00093E209A22FB32F08959A93A8
:104542008A936297602F212FCE010896E4ECFDE951
:1045520030E08C014AE050E00E94714ECE01EEEC58
:10456200FDE930E08C0148E050E00E94714E2032BB
:1045720011F02F3151F42395122FFE0170E0E60F56
:10458200F71F00810E94852F10C02F3158F4239508
:10459200122FFE01389670E0E60FF71F00810E948D
:1045A200852F03C001E20E94DB0D629689919991E9
:1045B20008958A93802F03C000E20E94DB0D082F2A
:1045C200802F8A950023C1F7899108950E948F4E0A
:1045D20080E005C00CE810E00E94C04B83958C334C
:1045E200C8F311E001E00E94852F05E21FE00E945E
:1045F200C04B0FE31FE00E94C04B07E2DADF0AE57F
:104602001FE00E94C04B07E61FE00E94C04B07E27A
:10461200D0DF02E81FE00E94C04B09E81FE00E94C1
:10462200C04B07E2C6DF04EA1FE00E94C04B02EB68
:104632001FE00E94C04B07E2BCDF0DEC1FE00E94AE
:10464200C04B0BED1FE00E94C04B07E2B2DF06EF4A
:104652001FE00E94C04B04E010E10E94C04B07E241
:10466200A8DF0FE110E10E94C04B0DE210E10E94B1
:10467200C04B07E29EDF08E410E10E94C04B06E552
:1046820010E10E94C04B07E294DF01E710E10E94B3
:10469200C04B0FE710E10E94C04B07E28ADF0AE934
:1046A20010E10E94C04B08EA10E10E94C04B07E2F1
:1046B20080DF03EC10E10E94C04B01ED10E10E948B
:1046C200C04B07E276DF0CEE10E10E94C04B0AEF0E
:1046D20010E10E94C04B07E26CDF05E111E10E948C
:1046E200C04B03E211E10E94C04B07E262DF0EE31E
:1046F20011E10E94C04B0CE411E10E94C04B07E2A1
:1047020058DF07E611E10E94C04B05E711E10E9464
:10471200C04B07E24EDF00E911E10E94C04B0EE9F7
:1047220011E10E94C04B07E244DF09EB11E10E9454
:10473200C04B07EC11E10E94C04B07E23ADF02EEE8
:1047420011E10E94C04B00EF11E10E94C04B07E251
:1047520030DF0BE012E10E94C04B09E112E10E943E
:10476200C04B07E226DF04E312E10E94C04B02E4E1
:1047720012E10E94C04B0DE512E10E94C04B08E716
:1047820012E10E94C04B03E912E10E94C04B0EEA03
:1047920012E10E94C04B09EC12E10E94C04B04EEF0
:1047A20012E10E94C04B0FEF12E10E94C04B0AE1DE
:1047B20013E10E94C04B05E313E10E94C04B00E5E8
:1047C20013E10E94C04B0BE613E10E94C04B06E8C6
:1047D20013E10E94C04BE8EDFCE000811181012B46
:1047E20029F406E214E10E94C04B04C007ED13E174
:1047F2000E94C04B05E714E10E94C04B80E001C05B
:1048020083958132F8F490E006C0A23019F4182F93
:10481200092F73DD9395933198F7182F092F00DD37
:10482200A02FAA23B9F3182F092F89DEA13069F727
:10483200182F092F13DDF801EB52F64F00810E9469
:10484200930EE8CFBADCEBEFF5E11491E2EFF5E17C
:1048520004910E94852F05ED19E00E94FF0EECEFF6
:10486200F5E11491E3EFF5E104910E94852FE8ED63
:10487200FCE0008111810E949D0EEDEFF5E11491A3
:10488200E4EFF5E104910E94852FE8EDFCE0008160
:10489200118120E030E040E052E060E070E00E94F0
:1048A200114E005010422F4F3F4F0E94EE0EE3E098
:1048B2000C94A04E0E94854EEF97EA97DA95BE01BE
:1048C20064527F4FE6EDFDE930E08B0141E250E0BA
:1048D2000E94714EA0E0BA2FBA2ECA2E24EF3FE0FA
:1048E200A9010E94B24D053511F40C94A22E1A2F83
:1048F2000B2F1ADC1A2F0B2F22DE9090E909009160
:104902005F09002319F000E1A02E02C00AE0A02EE8
:104912000E940C0F902F9B31D9F50E940C0F902F03
:104922009B3519F40E940C0F902F943421F4BB2371
:1049320089F0BA950FC0933411F4B3950BC091343A
:1049420021F4AA2339F0AA9505C0923419F4A032B1
:1049520008F4A395FE01E452FF4F0A2F10E0E00F86
:10496200F11F00810B1738F4FE01E452FF4FB0E053
:10497200EA0FFB1FB081BC1521F4AB1511F40C94A6
:104982003C2F1A2F0B2FD0DBCB2EBA2E0C943C2FA0
:10499200903209F044C01A2F0B2F42DC023011F082
:1049A2000C943C2F80E090E21A2F0B2F57DCF80179
:1049B200EB52F64F008111810827192700831183DA
:1049C200BB2329F58A2F02E0809F800100501E4FF1
:1049D200F801EB52F64F018105FD16C090E0FC0193
:1049E200E659F64F0081002379F014E2082F0E9465
:1049F200592F22E0829F20E0020E22E0121EF001D7
:104A0200EB52F64F008311830A2F0E94FA391A2FB4
:104A12000B2F73DC01E00093DA0C0C943C2F9D35D4
:104A220009F04CC01A2F0B2F8ADD1A2F0B2FF8DB3F
:104A32000130B9F41A2F0B2F11DCF801EB52F64FAB
:104A42000081039500831A2F0B2F08DCF801EB522B
:104A5200F64F00810E94930E01E00093DA0C0C9451
:104A62003C2F023011F00C943C2F1A2F0B2FF6DB47
:104A7200F801EB52F64F008111810F7F13700F3F47
:104A820023E0120711F40C943C2F1A2F0B2FE6DBB4
:104A9200F801EB52F64F008111810F5F1F4F008327
:104AA20011831A2F0B2F29DCBB2319F40A2F0E9422
:104AB200FA3901E00093DA0C0C943C2F9B3509F093
:104AC2004AC01A2F0B2F3BDD1A2F0B2FA9DB013007
:104AD200B9F41A2F0B2FC2DBF801EB52F64F00810B
:104AE2000A9500831A2F0B2FB9DBF801EB52F64F10
:104AF20000810E94930E01E00093DA0C0C943C2F8B
:104B0200023011F00C943C2F1A2F0B2FA7DBF80167
:104B1200EB52F64F008111810F7F1370012B11F4BC
:104B22000C943C2F1A2F0B2F99DBF801EB52F64F06
:104B32000081118101501040008311831A2F0B2F25
:104B4200DCDBBB2319F40A2F0E94FA3901E000933F
:104B5200DA0C0C943C2F9D3709F050C01A2F0B2F02
:104B62005FDB0130B9F41A2F0B2F78DBF801EB521F
:104B7200F64F00810A0D00831A2F0B2F6FDBF8010D
:104B8200EB52F64F00810E94930E01E00093DA0C83
:104B92000C943C2F023011F00C943C2F1A2F0B2F47
:104BA2005DDBF801EB52F64F008111810F7F13702C
:104BB2002FEF33E04A2D50E0241B350B0217130769
:104BC20010F00C943C2F8A2D90E01A2F0B2F46DB0D
:104BD200F801EB52F64F00811181080F191F008373
:104BE20011831A2F0B2F89DBBB2319F40A2F0E9482
:104BF200FA3901E00093DA0C0C943C2F9B3709F050
:104C02004CC01A2F0B2F0CDB0130B9F41A2F0B2FCB
:104C120025DBF801EB52F64F00810A1900831A2FA7
:104C22000B2F1CDBF801EB52F64F00810E94930E12
:104C320001E00093DA0C0C943C2F023011F00C943A
:104C42003C2F1A2F0B2F0ADBF801EB52F64F008193
:104C520011810F7F13702A2D30E00217130710F411
:104C62000C943C2F8A2D90E01A2F0B2FF7DAF801C3
:104C7200EB52F64F00811181081B190B008311833F
:104C82001A2F0B2F3ADBBB2319F40A2F0E94FA3991
:104C920001E00093DA0C0C943C2F74DA903360F04C
:104CA2009B3750F4092F0E94DB0D98A721E08E015B
:104CB200085D1F4F5DD905C020E08E01085D1F4FC2
:104CC20057D900E00883AE01485D5F4F9E012C5921
:104CD2003F4F8E010E940D1E902F992311F40C94C8
:104CE2003C2F28E935E08E010E94EB1D002351F094
:104CF20001E000935F09A0E0BA2F1A2F0B2F14DAFC
:104D02000C943C2F24E935E08E010E94EB1D002318
:104D120051F000E000935F09A0E0BA2F1A2F0B2F89
:104D220003DA0C943C2F2BE436E08E010E94EB1D3B
:104D3200002341F04BDCA0E0BA2F1A2F0B2FF4D93D
:104D42000C943C2F27E436E08E010E94EB1D0023D9
:104D520039F427EE35E08E010E94EB1D002391F01D
:104D6200EAEFF5E11491E1EFF5E104910E94852F5C
:104D72000E94300F2BDCA0E0BA2F1A2F0B2FD4D9B0
:104D82000C943C2F22E436E08E010E94EB1D00239E
:104D9200B1F0933021F002E0A3D90C943C2FFE0134
:104DA200FF9605A116A127A130A5B02FFE01FF96FF
:104DB20001A512A523A534A5A02F0C943C2F2DE309
:104DC20036E08E010E94EB1D002339F42BE336E01E
:104DD2008E010E94EB1D002349F1E8EDFCE02081E9
:104DE20031812F3700E03007E8F4E8EDFCE0008184
:104DF20011810F5F1F4F00831183CBDA002341F033
:104E0200E5DBA0E0BA2F1A2F0B2F8ED90C943C2F82
:104E1200E8EDFCE000811181015010400083118314
:104E22000C943C2F01E05CD90C943C2F24E336E037
:104E32008E010E94EB1D002339F422E336E08E013D
:104E42000E94EB1D002321F1E8EDFCE000811181BD
:104E5200012BD9F0E8EDFCE00081118101501040F6
:104E62000083118396DA002339F0B0DBA0E0BA2F79
:104E72001A2F0B2F59D9FFC7E8EDFCE000811181F1
:104E82000F5F1F4F00831183F6C701E029D9F3C7D3
:104E92002DE236E08E010E94EB1D002339F42BE255
:104EA20036E08E010E94EB1D002399F1923019F039
:104EB20002E016D9E0C7FE01FF9605A116A127A1BF
:104EC20030A5003840E0140740E0240740E03407F2
:104ED200E8F4E8EDFCE080819181FE01FF9605A1F6
:104EE20016A127A130A5E8EDFCE00083118351DA79
:104EF200002339F06BDBA0E0BA2F1A2F0B2F14D945
:104F0200BAC7E8EDFCE080839183B5C701E0E8D839
:104F1200B2C726E236E08E010E94EB1D0023D1F1DA
:104F2200923019F002E0DCD8A6C7FE01FF9605A177
:104F320016A127A130A5003840E0140740E024075D
:104F420040E0340720F5E8EDFCE080819181FE012C
:104F5200FF9605A116A127A130A5E8EDFCE000838C
:104F6200118317DA002371F0E8EDFCE0808391836E
:104F72002DDBA0E0BA2F1A2F0B2FD6D801E0009319
:104F8200DA0C79C7E8EDFCE08083918374C701E015
:104F9200A7D871C72AE536E08E010E94EB1D0023D7
:104FA200E1F00091DA0C002389F000E099D80E9428
:104FB2000C0F902F993519F0993709F05CC704E16D
:104FC20010E00E945C0C08E001BD55C704E110E04E
:104FD2000E945C0C08E001BD4EC721E236E08E0162
:104FE2000E94EB1D002319F10AE30E94DB0D20E071
:104FF2008E01085D1F4F0E94B91F002361F000E07F
:105002000DAB9E01285D3F4F05ED19E00E94D31DB7
:1050120001E00093DA0CEBEFF5E11491E2EFF5E138
:10502200049172D705ED19E00E94FF0E24C72EE10C
:1050320036E08E010E94EB1D002309F482C09130FC
:10504200A9F580E08F3108F016C702E0809F00E0EA
:10505200000E02E0101EF001EB52F64F018105FF37
:1050620023C090E0FC01E659F64F00810023E1F0F5
:1050720021E018E1082F0E947F4D14E2082F18D773
:1050820022E0829F20E0020E22E0121EF001EB528B
:10509200F64F00831183082F0E94FA39182F00E07F
:1050A2004EDA182F00E029D98395CCCF4424552419
:1050B200E92FF0E031974E165F060CF0DCC6FE01D8
:1050C200EC59FF4F042D10E0000F111F000F111FAC
:1050D200E00FF11F0081118122813381802F02E0D4
:1050E200809F00E0000E02E0101EF001EB52F64F2E
:1050F200018105FF24C0082F10E0F801E659F64FA0
:1051020000810023E1F021E018E1082F0E947F4D89
:1051120014E2082FCDD622E0829F20E0020E22E088
:10512200121EF001EB52F64F00831183082F0E94EA
:10513200FA39182F00E003DA182F00E0DED8439482
:10514200B6CF2AE136E08E010E94EB1D002309F45E
:1051520060C0913021F580E08F3108F08CC690E07C
:10516200FC01E659F64F00810023B9F020E018E176
:10517200082F0E947F4D02E0809F00E0000E02E0B7
:10518200101EF001EB52F64F018100620183182FCD
:1051920000E0D5D9182F00E0B0D88395DDCF4424A4
:1051A2005524E92FF0E031974E165F060CF063C6E6
:1051B200FE01EC59FF4F042D10E0000F111F000FEC
:1051C200111FE00FF11F0081118122813381802F95
:1051D200082F10E0F801E659F64F00810023B9F0DC
:1051E20020E018E1082F0E947F4D02E0809F00E03E
:1051F200000E02E0101EF001EB52F64F0181006238
:105202000183182F00E09BD9182F00E076D8439431
:10521200C7CF22E136E08E010E94EB1D002309F484
:1052220066C0913009F048C00091FE0C1091FD0C4F
:10523200011709F020C608EC10E00E945C0C0E94E5
:10524200C320EAEFF5E11491E1EFF5E104915CD6B8
:1052520012E206E60E945A4D0E94930E00E20E945C
:10526200DB0D13E206E60E945A4D0E94930E00E205
:105272000E94DB0D14E206E60E945A4D0E94930E34
:105282000CE20E94DB0D12E205E60E945A4D0E94DA
:10529200930E00E20E94DB0D13E205E60E945A4DD6
:1052A2000E94930E00E20E94DB0D14E205E60E94CA
:1052B2005A4D0E94930EB8CF923009F0DCC580E0BF
:1052C20007C000E090E0FC01E455F24F00838395B3
:1052D2008F31B8F3FE01FF9605A116A127A130A5D3
:1052E2000093D70C07E115E10E94C04BC4C52DE025
:1052F20036E08E010E94EB1D002339F423E936E0EB
:105302008E010E94EB1D0023C1F0FE01FF9605A154
:1053120016A127A130A5923021F002E00E9471204F
:10532200AAC5083020F004E00E947120A4C50093B1
:10533200E90901E00093DA0C9EC52EE836E08E0101
:105342000E94EB1D002399F1933021F002E00E94AC
:10535200712091C5FE01FF9605A116A127A130A5D6
:10536200802FFE01FF9601A512A523A534A5902F3B
:10537200983010F4883020F004E00E9471207BC540
:105382000AE30E94DB0D082F0E94930E0DE20E9499
:10539200DB0D0EE30E94DB0D092F0E94930E182FE6
:1053A200092F0E94102001E00093DA0C64C52DE75A
:1053B20035E08E010E94EB1D002341F428E735E021
:1053C2008E010E94EB1D002309F488C0933020F067
:1053D20002E00E9471204FC5913019F40091E90951
:1053E20006C0FE01FF9605A116A127A130A5073030
:1053F20020F004E00E9471203EC5E8EDFCE020812F
:105402003181232B41F41091E909133020F004E09B
:105412000E94712030C5923039F417E00E941020AA
:1054220001E00093DA0C19C09130A1F40091E9096E
:10543200073080F417E00091E9090E941020E5EDA1
:10544200F9E004890395048B0E94DE2001E00093B9
:10545200DA0C03C004E00E947120E8EDFCE0008158
:105462001181012B09F007C50091E909013029F0EA
:105472000091E909023009F0FEC400E410E020E8DE
:1054820030E040EC50E080E01EC062E0869F020EF9
:10549200131EF001EB52F64F2080318062E0869FAE
:1054A200000E111EF001EB52F64F60817181261A37
:1054B200370A62E0869F040E151EF001EB52F64F8A
:1054C2002082318283958F3100F30E94C32003E052
:1054D2000E94712002E00E944320CDC427E836E0FA
:1054E2008E010E94EB1D002339F42BE036E08E0181
:1054F2000E94EB1D0023E9F1923029F5FE01FF968F
:1055020005A116A127A130A5802F873020F004E045
:105512000E947120B0C40091E909801770F4E5ED92
:10552200F9E004890A95048B0E94DE2006C0182F38
:105532001395082F0E94102083958630C0F301E056
:105542000093DA0C98C4913009F095C40091E909EE
:10555200013058F0E5EDF9E004890A95048B0E94C8
:10556200DE2001E00093DA0C86C404E00E94712080
:1055720082C420E836E08E010E94EB1D002339F43C
:105582002EE736E08E010E94EB1D002389F1FE0119
:10559200FF9605A116A127A130A5802F923021F0F8
:1055A20002E00E94712067C4873020F004E00E946C
:1055B200712061C406E0402E06C0142D1A95042DF8
:1055C2000E9410204A948415C0F317E0082F0E940D
:1055D20010200091E909801738F4E5EDF9E004891B
:1055E2000395048B0E94DE2001E00093DA0C43C491
:1055F2002DEB35E08E010E94EB1D002379F09230F5
:1056020048F0FE01FF9605A116A127A130A50E9430
:10561200134131C401E00E9413412DC42FE435E04F
:105622008E010E94EB1D002341F42DE435E08E0132
:105632000E94EB1D002309F461C0FE01FF9605A143
:1056420016A127A130A5402E923021F002E00E943F
:10565200712011C407E0401620F004E00E9471207E
:105662000AC499E580E01DC0082F10E0F801E65950
:10567200F64F00810023A1F0042D10E040E450E039
:105682000E94D04D22E0829F000E111E00E4000E07
:1056920000E0101EF001EB52F64F018106FD9EE480
:1056A20083958F3108F30091E909401640F099354E
:1056B20031F400E00E9471200E940C0F902F993566
:1056C20019F0993709F0D7C3EFEFF5E11491E6EF3E
:1056D200F5E1049119D4042D0E94930E07E00E9473
:1056E2004320142D07E00E94102080E08F3108F043
:1056F200C2C3082F0E94FA398395F8CF29E736E012
:105702008E010E94EB1D002309F4BAC0E8EDFCE013
:1057120040805180913061F4E8EDFCE0008111811C
:1057220020E030E0FE01FF9605A316A327A330A7D1
:10573200E4EDFDE020813181273302E0300738F0CB
:1057420023E333E012E20EEF0E94874D06C02FEFF3
:1057520033E012E20EEF0E94874D00E010E0E8ED28
:10576200FCE00083118380E00CC022E0829F20E0F5
:10577200020E22E0121EF001EB52F64F008311835B
:1057820083958F3100F590E0FC01E659F64F0081D8
:105792000023B1F318E1082F0E945A4D013021F481
:1057A2001EE1082F85D303C014E2082F81D30030F5
:1057B20020E41207D1F60DED1DE00E94C04B082F28
:1057C2000E94930EDDCFE8EDFCE040825182FE01A3
:1057D200FF9605A116A127A130A5A6D407C001E016
:1057E2000093DB0C05EF1DE00E94C04B0091DD0C25
:1057F2000023A1F00091FE0C1091FD0C0117B1F3F2
:105802000E940C0F0B3159F30D3081F702E0009327
:10581200DB0C0CEF1DE00E94C04BE8CF07E115E165
:105822000E94C04B04EF11E00E945C0C80E00CC0AF
:1058320022E0829F20E0020E22E0121EF001EB52D3
:10584200F64F0083118383958F31B0F490E0FC0111
:10585200E659F64F00810023B1F31EE1082F28D349
:10586200003020E4120721F70DED1DE00E94C04B2D
:10587200082F0E94930EE7CF07E00E944320FBC24D
:1058820025E736E08E010E94EB1D002309F457C084
:10589200923051F4FE01FF9605A116A127A130A571
:1058A200003024E0120720F002E00E947120E3C2DF
:1058B2001A2F0B2F0E94A0221A2F0B2F0E941121A8
:1058C2000130E9F4FE01FF9605A116A127A130A53A
:1058D200802F1A2F0B2F0E942F21F801EB52F64F27
:1058E20080831A2F0B2F0E942F21F801EB52F64FC3
:1058F20000810E94930E01E00093DA0CBCC20230D8
:1059020009F0B9C2FE01FF9605A116A127A130A593
:10591200C8011A2F0B2F0E942F21F801EB52F64FCC
:10592200808391831A2F0B2F0E947E21BB2319F4AF
:105932000A2F0E94FA3901E00093DA0C9CC22EE68B
:1059420036E08E010E94EB1D002341F42CE636E086
:105952008E010E94EB1D002309F443C1BE01605F6A
:105962007F4FE7EFFDE930E08B0148E150E00E9414
:10597200714E923071F4FE01FF9605A116A127A186
:1059820030A5073040E0140740E0240740E0340728
:1059920020F002E00E9471206EC201E00093DA0C56
:1059A200FE01FF9605A116A127A130A5102F07E041
:1059B2000E94102040E452EE60E070E080E03AC0C5
:1059C20002E0809F8001212F220F220B322F040F31
:1059D200151F261F371F0F5F1F4F2F4F3F4FF80115
:1059E200322F3BBF069000E00BBF302C222402E096
:1059F200809F8001212F220F220B322F040F151FAF
:105A0200261F371FF801322F3BBF0690202D00E0E2
:105A12000BBF30E0220D331D2F7F3370FE01E55C9A
:105A2200FE4F082F10E0000F111FE00FF11F20831F
:105A3200318383958F3120F2FE01FF9605A116A1D5
:105A420027A130A540E450E00E94D04D005C1F4FDA
:105A520080E026C022E0829F000E111E21E0020E8D
:105A620020E0121EF001EB52F64F508140E022E09E
:105A7200829F000E111EF001EB52F64F208130E0A2
:105A8200240F351F2F7F3370FE01E350FF4F482F45
:105A920050E0440F551FE40FF51F20833183839597
:105AA2008F31C0F280E068C0FE01E55CFE4F082F36
:105AB20010E0000F111FE00FF11F208131812F7FB5
:105AC20033708E0103501F4FFE01709690E0E80F75
:105AD200F91F408150E0440F551F040F151FE02F9E
:105AE200F12F008111810F7F1370201B310B8E016A
:105AF200055C1E4FFE01709690E0E80FF91F408191
:105B020050E0440F551F040F151FE02FF12F0081A5
:105B120011810F7F1370020F131F22E0829F20E07A
:105B2200020E22E0121EF001EB52F64F00831183A7
:105B32008E0103501F4FFE01709690E0E80FF91F8F
:105B4200208130E0220F331F020F131FE02FF12FAD
:105B52000081118100701C7F22E0829F20E0020EF2
:105B620022E0121EF001EB52F64F20813181202BF0
:105B7200312B2083318383958F3138F590E0FC01FE
:105B8200E659F64F00810023B1F3FE01709690E0D2
:105B9200E80FF91F00810F3F09F086CFFE01E350A5
:105BA200FF4F082F10E0000F111FE00FF11F0081BF
:105BB200118122E0829F20E0020E22E0121EF001FB
:105BC200EB52F64F00831183D6CF07E00E944320A9
:105BD20080E08F3108F04FC1082F0E94FA39839577
:105BE200F8CF28E636E08E010E94EB1D0023C1F0BB
:105BF20000E00E9471200E940C0F093519F009374C
:105C020009F039C10E9462220E94E722A0E0BA2F65
:105C12001A2F0B2F0E94952001E00093DA0C2BC162
:105C220023E636E08E010E94EB1D002341F42FE5AE
:105C320036E08E010E94EB1D002309F418C110E02A
:105C420088242FEF3FE0A9010E94B24D22EF3FE0EE
:105C5200A9010E94BE4D01E12FEF3FE0A9010E9480
:105C6200BE4D80E090E006C0FC01EB52F64F008191
:105C7200100F0196803002E09007B0F30091F40912
:105C8200011B0A950093F4090EE20E94DB0D80E0ED
:105C920090E00BC0FC01EB52F64F00819C012050BA
:105CA200384FA9010E94BE4D0196803002E0900754
:105CB20088F30091130C20E03AE0A9010E94BE4D46
:105CC2000091140C21E03AE0A9010E94BE4D80E04F
:105CD20090E001C00196803002E0900770F49C01D0
:105CE2002050384FA9010E94B24DFC01EB52F64FF1
:105CF2001081011779F388248394E8EDFCE0008198
:105D0200118125EF3FE0A9010E94BE4D882009F0D4
:105D120075C025EF3FE0A9010E94B24DE8EDFCE01D
:105D220020813181021709F069C00AEA24EF3FE0BD
:105D3200A9010E94BE4D08E001BD04EF11E00E94DE
:105D42005C0C25EF3FE0A9010E94B24D10E0E8EDA6
:105D5200FCE000831183E8EDFCE0008111810F7FFC
:105D620010700083118388240FEF24EF3FE0A90114
:105D72000E94BE4DE8EDFCE00081118120E030E0A0
:105D820040E052E060E070E00E94114E28013901CB
:105D920000E0400E00EE501E00E0601E00E0701EAB
:105DA20080E090E001C00196803002E09007C0F4EC
:105DB2009C012050384FA9010E94B24D602F8C01E6
:105DC20020E030E0040D151D261D371DF801322F8D
:105DD2003BBF069000E00BBF601529F302E0802E66
:105DE20020E03AE0A9010E94B24D0093130C21E099
:105DF2003AE0A9010E94B24D0093140C8820F9F4F4
:105E02000E94CA210091EA09002361F0E8EDFCE05A
:105E1200008111812091EA0930E020503F4FA90111
:105E22000E94BE4D07E115E10E94C04B0E94E7228D
:105E3200A0E0BA2F1A2F0B2F0E94952009C005ED62
:105E42001DE00E94C04B00E3800E082D0E94DB0D76
:105E520000E00093DA0C22EF3FE0A9010E94B24D6C
:105E62002FEF3FE0A9010E94BE4DAD9804C008EE9D
:105E72001DE00E94C04B0091E909091599F00091BB
:105E8200E909013F20F000E00093E90907C0009111
:105E9200E909083018F007E00093E9090E94DE20C2
:105EA2009090E9091A2F0B2F0E94A0220C948924AA
:105EB2009A938A93802F082F0E94694D0F3F2FEFEC
:105EC200120719F400E012E01CC0E8EDFCE02081AA
:105ED2003181232B51F090E0880F991FFC01EB5682
:105EE200F64F20813181021B130B212F27FF03C0A4
:105EF20000E010E006C0003024E0120710F00FEFBF
:105F020013E08991999108959A938A93902F812F02
:105F120002E00E94DB0D0BE10E94DB0D0BE50E940B
:105F2200DB0D8A3038F0082F4AE00E94C24D005D36
:105F32000E94DB0D082F4AE00E94C24D042F005D33
:105F42000E94DB0D0BE30E94DB0D9A3038F0092F23
:105F52004AE00E94C24D005D0E94DB0D092F4AE01B
:105F62000E94C24D042F005D0E94DB0D06E60E94D6
:105F7200DB0D8991999108959A938A93FA93EA9302
:105F82003A922A921A920A927A936A935A934A936B
:105F92003A932A931A930A938FB79BB700E00BBFE9
:105FA20078940091DD0C002349F00091DC0C002371
:105FB20021F004E20E94DB0D01C0CED0EFEEFCE046
:105FC200008111810F5F1F4F0083118300911B0E0F
:105FD200102F139510931B0E0F70002309F06EC043
:105FE200E1EFFCE000811181012B41F0E1EFFCE0E7
:105FF2000081118101501040008311830091EE0C49
:10600200002349F0EEEEFCE000810A95008308E0EF
:1060120015B3102715BBAA9AA99A24B135B10091DC
:10602200DC0D10E003701070000F111FF801EC522C
:10603200F24F20833183ECEDFDE000810395008374
:10604200037007B900911C0E102F139510931C0EAC
:106052000770002399F5EBECFDE0008103950083C6
:106062000E946F43879B2AC0969B28C00091E80C30
:10607200002321F500919A000F7700939A00959AD8
:1060820096980FE113E001501040E9F700C00000BC
:1060920000919B00102F17FF0AC000919C0005354C
:1060A20031F404E110E00E945C0C08E001BD969A14
:1060B200959800919A00006800939A00EDEDFDE03A
:1060C200008107FF0CC000911B0E002311F4A89859
:1060D20015C000911B0E083089F4A89A0FC00091D8
:1060E2001B0E1091DD0D1023112341F40091DD0DE3
:1060F200002321F001E015B3102715BB00E0009347
:10610200100D9BBF8FBF0991199129913991499126
:106112005991699179910990199029903990E99151
:10612200F9918991999118959A938A93C80120E0DF
:1061320030E010E20EEF0E94874DEAEEFCE0808331
:10614200918301E00093E90C0093DD0C00E00093E1
:10615200DB0C8991999108950E94844E24970091B5
:10616200E90C002309F44DC000E000935E1000E04A
:1061720010E0E4E5F0E100831183E2E5F0E1008361
:106182001183E6E5F0E10083118300E00093A50CA2
:1061920003E000935C10CC2431C002E0C09E800179
:1061A20000501E4FF801EB52F64F208131810C2D29
:1061B20010E0000F111FF801E75DF04F20833183DB
:1061C20000E010E02C2D30E0220F331FF901E151E5
:1061D200F04F008311832C2D30E0220F331FF90181
:1061E200EF5DF14F008311832C2D30E0220F331F1E
:1061F200F901E355F04F00831183C3940FE1C016F8
:1062020060F2E2E5F0E100811181E4E5F0E1208154
:1062120031810217130708F00CC3E2E5F0E10081B7
:1062220011810F5F1F4F00831183E7EDFCE00081B6
:1062320000FF86C0EFEEFCE00081118103700023B5
:1062420009F059C002E20093950703E00093960714
:1062520022E012E006E60E949C4A002331F00091FF
:106262001C0810911D0890911E0800915F10000FEC
:1062720000935F10EFE5F0E1008101FF08C09B3061
:1062820068F0EFE5F0E100810160008307C093331D
:1062920028F0EFE5F0E100810160008302E2009363
:1062A200950703E00093960722E012E005E60E94BC
:1062B2009C4A002331F000911C0810911D08809126
:1062C2001E0800916010000F00936010E0E6F0E1FC
:1062D200008101FF08C08B3098F1E0E6F0E1008117
:1062E200016000832DC0833358F1E0E6F0E10081C4
:1062F2000160008325C0EFEEFCE000811181037094
:10630200013061F408E20093950704E000939607D8
:1063120022E012E007E60E949C4A12C0EFEEFCE087
:10632200008111810370023059F404E30093950750
:1063320004E00093960722E012E007E60E949C4ADE
:1063420000915C10033009F474C280E00CE190E02B
:10635200FC01EB56F84F0083839504E090E0FC01CA
:10636200EB56F84F00838395CC244CC001E010E03B
:106372002C2D30E0205E3F4FF901EA56F34F408169
:1063820042954F700E94E04D90E0FC01EB56F84FB1
:106392000083839501E010E02C2D30E0205E3F4F1A
:1063A200F901EA56F34F40814F700E94E04D90E0B0
:1063B200FC01EB56F84F0083839502E0C09E00E09B
:1063C200000E02E0101EF001EB52F64F0081118127
:1063D20090E0FC01EB56F84F0083839502E0C09EEB
:1063E20000E0000E02E0101EF001EB52F64F0081B9
:1063F2001181012F10E090E0FC01EB56F84F008371
:106402008395C3940FE1C01608F00EC2DD24F60195
:10641200E659F64F00810023A1F300915C1000239E
:1064220009F092C00C2D10E0000F111FF801E55980
:10643200F04F008111812C2D30E0220F331FF90122
:10644200E355F04F20813181021B130B212F220FC4
:10645200220B322FE2E5F0E14081518160E070E0F1
:106462000E94114EE4E5F0E14081518160E070E06C
:106472000E945B4E2C2D30E0220F331FF901E355B1
:10648200F04F40815181400F511F2C2D30E0220FDF
:10649200331FF901E151F04F408351832C2D30E03D
:1064A200220F331FF901E355F04F208131811595F9
:1064B2000795020F131F212F220F220B322FE2E525
:1064C200F0E14081518160E070E00E94114E40E9AC
:1064D20050E060E070E00E94114E4FE050E060E05A
:1064E20070E00E945B4E012F122F232F330F330BCC
:1064F2002595179507952C2D30E0220F331FF901B2
:10650200EB55F14F008311830C2D10E0000F111F8A
:10651200F801E951F14F208131810C2D10E0000F7B
:10652200111FF801EB55F14F00811181020F131F6A
:1065320022E0C29E20E0020E22E0121EF001EB5287
:10654200F64F0083118310C100915C10013009F0F5
:1065520046C00C2D10E0000F111FF801E951F14F58
:10656200A081B1810C2D10E0000F111FF801ED592F
:10657200F14F00811181212F220F220B322FE2E5F0
:10658200F0E14081518160E070E00E94114EE4E54B
:10659200F0E14081518160E070E00E945B4E0A0FA1
:1065A2001B1F22E0C29E20E0020E22E0121EF0011A
:1065B200EB52F64F008311830C2D10E0000F111FD8
:1065C200F801E559F04F208131810C2D10E0000FC8
:1065D200111FF801E151F04F20833183C5C0DD2442
:1065E200F601EF5CFF4E0081002309F078C00C2D0C
:1065F20010E0000F111FF801E355F04F00811181E7
:10660200119501951040212F220F220B322FE2E526
:10661200F0E14081518160E070E00E94114EE4E5BA
:10662200F0E14081518160E070E00E945B4E2C2DD0
:1066320030E0220F331FF901E355F04F40815181C1
:10664200400F511F2C2D30E0220F331FF901E15171
:10665200F04F408351832C2D30E0220F331FF9017C
:10666200E951F14FA081B1812C2D30E0220F331F6F
:10667200F901E355F04F2081318115950795020FFD
:10668200131F212F220F220B322FE2E5F0E140816E
:10669200518160E070E00E94114E40E950E060E0FC
:1066A20070E00E94114E4FE050E060E070E00E9406
:1066B2005B4E012F122F232F330F330B2595179586
:1066C20007950A0F1B1F22E0C29E20E0020E22E065
:1066D200121EF001EB52F64F0083118345C00C2DC0
:1066E20010E0000F111FF801E951F14FA081B181B3
:1066F2000C2D10E0000F111FF801ED59F14F008130
:106702001181212F220F220B322FE2E5F0E140818D
:10671200518160E070E00E94114EE4E5F0E14081B9
:10672200518160E070E00E945B4E0A0F1B1F22E065
:10673200C29E20E0020E22E0121EF001EB52F64F42
:10674200008311830C2D10E0000F111FF801E55991
:10675200F04F208131810C2D10E0000F111FF80144
:10676200E151F04F2083318302E0C09E00E0000E31
:1067720002E0101EF001EB52F64F018107FF0EC03E
:1067820000E010E022E0C29E20E0020E22E0121E93
:10679200F001EB52F64F008311831CC002E0C09E51
:1067A20000E0000E02E0101EF001EB52F64F2081D5
:1067B2003181203004E0300768F00FEF13E022E06F
:1067C200C29E20E0020E22E0121EF001EB52F64FB2
:1067D2000083118390E0FC01EB56F84FC082839551
:1067E200E7EDFCE0008100FFC1CD00915F100F3F9B
:1067F20019F004E1C01649F0009160100F3F09F44E
:10680200B5CD05E1C01609F0B1CD00E890E0FC017C
:10681200EB56F84F0083839500E890E0FC01EB56BD
:10682200F84F00838395C9CD282F13E80EEF0E94FD
:10683200214A00915E10002321F000E00093DD0C5C
:10684200D4C5E2E5F0E100811181E4E5F0E12081C7
:1068520031810217130708F4C8C500E010E0E2E531
:10686200F0E100831183CC2427C002E0C09E00E047
:10687200000E02E0101EF001EB52F64F2081318132
:106882000C2D10E0000F111FF801E951F14F208388
:1068920031830C2D10E0000F111FF801E151F04F70
:1068A200208131810C2D10E0000F111FF801E355FA
:1068B200F04F20833183C3940FE1C016B0F20091F0
:1068C2005C10002309F09FC001E000935C10E8E532
:1068D200F0E100811181EAE5F0E120813181220FAE
:1068E200331F021B130BE4E5F0E100831183CC2478
:1068F20046C00C2D10E0000F111FF801EF5DF14FA3
:10690200808191810C2D10E0000F111FF801EB55D1
:10691200F14F00811181801B910B0C2D10E0000FB3
:10692200111FF801E559F04F00811181212F220F2B
:10693200220B322FEAE5F0E14081518160E070E004
:106942000E94114E4CE050E060E070E00E94114E57
:1069520045E050E060E070E00E945B4E012F122F94
:10696200232F330F330B801B910B0C2D10E0000FE4
:10697200111FF801ED59F14F80839183C3940FE108
:10698200C01608F0D6C0DD24F601EF5CFF4E008190
:10699200013009F0AECF0C2D10E0000F111FF801ED
:1069A200EF5DF14F008111812C2D30E0220F331F5A
:1069B200F901EB55F14F20813181021B130B212F7D
:1069C200220F220B322FE4E5F0E14081518160E099
:1069D20070E00E94114EE8E5F0E140815181EAE564
:1069E200F0E160817181461B570B60E070E00E940C
:1069F2005B4E2C2D30E0220F331FF901ED59F14F80
:106A020000831183BBCF00915C100130D1F502E00D
:106A120000935C10EAE5F0E100811181E4E5F0E128
:106A220000831183CC240FE1C01608F082C00C2D24
:106A320010E0000F111FF801EF5DF14F208131814D
:106A42000C2D10E0000F111FF801ED59F14F0081DC
:106A52001181201B310B0C2D10E0000F111FF801CA
:106A6200EB55F14F00811181201B310B0C2D10E0F1
:106A7200000F111FF801ED59F14F20833183C394A8
:106A8200D2CF00915C100230B1F4E6E5F0E1008172
:106A92001181012B61F003E000935C10E6E5F0E167
:106AA20000811181E4E5F0E10083118342C000E03E
:106AB20000935C103EC000915C100330D1F5CC24F1
:106AC20032C002E0C09E00E0000E02E0101EF001A3
:106AD200EB52F64F208131810C2D10E0000F111F77
:106AE200F801E75DF04F2083318300E010E02C2DA8
:106AF20030E0220F331FF901E151F04F008311837F
:106B02002C2D30E0220F331FF901EF5DF14F00838E
:106B120011832C2D30E0220F331FF901E355F04F82
:106B220000831183C3940FE1C01658F200E0009372
:106B32005C1000915C10002309F057C4EDE5F0E110
:106B420000810395008300915D101091AA0C01173A
:106B520028F40091E90C002309F4DFC00091E90C4C
:106B6200002399F5EAEEFCE000811181ECEEFCE0F5
:106B7200008311830091A50C002329F0E6E9FCE0D3
:106B820007850A9507870091A50C0023F1F400916F
:106B9200DB0C013039F400E010E0EAEEFCE00083A7
:106BA200118313C00091DB0C023041F40091B00C50
:106BB20010E0EAEEFCE00083118307C00091AF0C05
:106BC20010E0EAEEFCE000831183EAEEFCE00081D3
:106BD2001181012B21F401E000935E109EC000E0C0
:106BE2000093E90CE8EDFCE000811181EAEEFCE0A3
:106BF200208131810217130741F500E010E020E007
:106C020030E0EDE1FEE000831183228333830091C3
:106C1200A50C002309F053C0ADE0B0E0A03400E0C1
:106C2200B00708F04CC0EDE1FEE000811181228145
:106C320033810A0F1B1FF801EB52F64F0081FD0151
:106C4200EA56F34F00831196E9CFEAEEFCE00081A9
:106C5200118120E030E0322F212F102F00E0110FA0
:106C6200221F331F005010422F4F3F4FEDE1FEE035
:106C720000831183228333830091A50C0023F9F44E
:106C8200ADE0B0E018C0EDE1FEE0408151816281EB
:106C920073818D0120E030E0040F151F261F371F7E
:106CA200F801322F3BBF069000E00BBFFD01EA5610
:106CB200F34F00821196A03400E0B00720F3EDE11B
:106CC200FEE00081118122813381005C1F4F2F4F32
:106CD2003F4F00831183228333830091AA0C083033
:106CE20020F40091AA0C002381F40BE01DE00E9425
:106CF200C04BEAEEFCE0008111810E94E20E0DE53C
:106D02000E94DB0D01E000935E100091A50C0023B0
:106D120009F428CF00E000935D10A0E0B0E020C0AD
:106D2200EDE1FEE00081118122813381A801B901E8
:106D32004F5F5F4F6F4F7F4FEDE1FEE04083518326
:106D420062837383F801322F3BBF069000E00BBFD2
:106D52008D01005C1D4FF801EB52F64F0082119637
:106D6200A03400E0B00758F5E8EDFCE000811181A5
:106D7200EAEEFCE0208131810217130789F6EDE18A
:106D8200FEE00081118122813381F801EB52F64F3E
:106D920020818D01005C1D4FF801EB52F64F2083DC
:106DA200EDE1FEE000811181228133810F5F1F4FEF
:106DB2002F4F3F4F0083118322833383D0CF009123
:106DC2005D100395EAEEFCE0808191811091AA0C9E
:106DD200011708F456C00091DB0C013039F400E0D1
:106DE20010E0EAEEFCE00083118312C00091A50CD2
:106DF200023028F0EAEEFCE08081918109C0009126
:106E0200DB0C023019F48091B00C02C08091AF0CFF
:106E120090E0E8EDFCE0008111818017910759F4C0
:106E220000E410E020E030E0EDE1FEE000831183B9
:106E32002283338326C0882379F4EDE1FEE00081CA
:106E42001181228133810054104020403040008360
:106E520011832283338315C0082F10E020E030E035
:106E6200322F212F102F00E0110F221F331F005C41
:106E72001F412F4F3F4FEDE1FEE00083118322833C
:106E82003383A0E0B0E01BC0EDE1FEE04081518120
:106E9200628173818D0120E030E0040F151F261FEF
:106EA200371FF801322F3BBF069000E00BBF8D0168
:106EB20000581D4FF801EB52F64F00821196A03494
:106EC20000E0B007D0F4E8EDFCE00081118180170A
:106ED200D9F6EDE1FEE000811181228133810A0FB2
:106EE2001B1FF801EB52F64F20818D0100581D4FF8
:106EF200F801EB52F64F2083E1CF00915E100023A0
:106F020009F073C20091530C10E045E00E94E04D7D
:106F12004091AC0C50E00E94EC4DE6E5F0E10083BC
:106F220011830091540C1091AC0C019F800145E03B
:106F32000E94E64DD8010A2F0B2B11F4A1E0B0E01C
:106F420020E030E0CC240EC00C2D10E0000F111F09
:106F5200F801EF5DF14F008111812017310708F42C
:106F62009801C3940FE1C01608F0F7C0DD24F601C2
:106F7200E659F64F00810023A1F30C2D10E0000F1B
:106F8200111FF801E75DF04F4081518102E0C09E80
:106F920000E0000E02E0101EF001EB52F64F4083BB
:106FA20051830C2D10E0000F111FF801E951F14F30
:106FB2004083518300E010E04C2D50E0440F551FF8
:106FC200FA01EB55F14F0083118302E0C09E00E409
:106FD200000E02E0101EF001EB52F64F008111810B
:106FE2004C2D50E0440F551FFA01EB56F64F6081CD
:106FF2007181DD24F601E455F24F4081542F550F83
:10700200550B460F571F040F151F412F47FF03C093
:1070120000E010E006C0003044E0140710F00FEF6B
:1070220013E04C2D50E0440F551FFA01E75DF04F7D
:1070320040815181B801641B750B4C2D50E0440F07
:10704200551FFA01EF5DF14F608371834C2D50E0C3
:10705200440F551FFA01E75DF04F608171814C2D9D
:1070620050E0440F551FFA01E75DF04F0083118392
:1070720042E0C49E40E8040E42E0141EF001EB52CE
:10708200F64F208031804C2D50E0440F551FFA01FD
:10709200EB56F64F00801180020C131CDD24F60122
:1070A200E455F24F4081542F550F550B400D511DA1
:1070B200052E07FE03C040E050E006C04030E4E089
:1070C2005E0710F04FEF53E06017710718F40417D2
:1070D200150730F00617170728F44017510710F468
:1070E20000E001C001E0002391F4E6E5F0E1008157
:1070F2001181012B61F400915D1010E0E091AA0C66
:10710200F0E031970E171F074CF0882339F400E0A6
:10711200DD24F601EF5CFF4E008306C001E0DD24B2
:10712200F601EF5CFF4E00830C2D10E0000F111FE3
:10713200F801EF5DF14F4081518155230AF004CFF0
:107142000C2D10E0000F111FF801EF5DF14F0081CF
:10715200118111950195104000CF890148E250E05C
:107162000E94D04DC8018D0143E050E00E94D04DF5
:10717200A8018C010E94EC4DE8E5F0E10083118347
:107182000091AE0C10E0EAE5F0E100831183EAE53C
:10719200F0E100811181000F111FE8E5F0E120818B
:1071A200318102171307E8F1E7E6F9E0008102FFF7
:1071B20013C00BE50E94DB0D00915D100E94C40D0F
:1071C2000CE20E94DB0DE8E5F0E1008111810E94F2
:1071D200E20E0DE50E94DB0DE8E5F0E10081118190
:1071E200012B39F400E010E0EAE5F0E100831183BD
:1071F20018C0E8E5F0E100811181015010401695B8
:107202000795EAE5F0E100831183EAE5F0E1008108
:107212001181012B31F400E010E0E8E5F0E1008398
:107222001183E8E5F0E10081118120E030E0000FF8
:10723200111F221F331FEAE5F0E180819181A0E056
:10724200B0E0880F991FAA1FBB1F081B190B2A0B3E
:107252003B0B48015901880C991CAA1CBB1C880EC7
:10726200991EAA1EBB1E000F111F221F331F088367
:1072720019832A833B83082D09290A290B2929F41A
:107282009924AA24BB2488248394088119812A8101
:107292003B81012B022B032B41F401E010E020E0A3
:1072A20030E0088319832A833B83CC2442C004192B
:1072B200150926093709A401B5010E945B4E2C2D40
:1072C20030E0220F331FF901E559F04F008311839B
:1072D2000C2D10E0000F111FF801E559F04F20812D
:1072E2003181203004E030075CF00FEF13E02C2DE9
:1072F20030E0220F331FF901E559F04F008311836B
:107302000C2D10E0000F111FF801E559F04F2081FC
:10731200318121300CEF30075CF401E01CEF2C2DA1
:1073220030E0220F331FF901E559F04F008311833A
:10733200C3940FE1C01608F050C00C2D10E0000FEE
:10734200111FF801E355F04F00811181212F220F07
:10735200220B322FAC01BD010E94114E28013901CE
:107362000C2D10E0000F111FF801EF5DF14F0081AD
:107372001181212F220F220B322F0801190140E027
:107382005AE060E070E0800191010E94114E080114
:1073920019014CE050E060E070E0800191010E9430
:1073A2005B4EDD24F601EF5CFF4E4081442309F081
:1073B2007ECF0419150926093709488159816A8146
:1073C2007B810E945B4E2C2D30E0220F331FF9018E
:1073D200E559F04F008311837BCFEAE5F0E10081AC
:1073E2001181E4E5F0E1008311832496EEE00C9430
:1073F200954E0E948C4E402E5524F201E659F64FCE
:107402000081002309F47EC002E0409E800100500A
:107412001E4FF801EB52F64F018105FF06C020E036
:1074220018E1042D0E947F4D6DC0E8EDFCE0008163
:107432001181012BC9F002E0409E00E0000E02E043
:10744200101EF001EB52F64F008111810F7F137075
:10745200242D30E0220F331FF901EB56F64FA081A5
:10746200B181A00FB11F0DC002E0409E00E0000EEE
:1074720002E0101EF001EB52F64FA081B181AF7F06
:10748200B3700B2F07FF03C0A0E0B0E006C0A0302E
:1074920004E0B00710F0AFEFB3E014E2042D0E9455
:1074A200694D0F3F23E0120758F4A017B10720F4EB
:1074B2000A1B1B0BC80106C0CD01801B910B02C029
:1074C20008E010E09695879596958795883000E0BC
:1074D200900710F488E090E00EE1009395070A2FE0
:1074E20000939607AB2FB0E0A0939707082F009365
:1074F2009807892F90E08093990725E013E0042DE7
:107502000E949C4AE6E00C949D4E0E948E4ED80149
:107512000091DD0C002309F041C00A2F0B2BF1F181
:10752200A03800E0B007D0F500E010E0E8EDFCE0A4
:107532000083118380E00BC022E0829F90012050E3
:107542003E4FF901EB52F64F0083118383958F3141
:1075520010F590E0FC01E659F64F00810023B1F3EB
:1075620018E1082F0E945A4D013029F41EE1082F1C
:107572000E94592F04C014E2082F0E94592F003094
:1075820020E41207C9F60DED1DE00E94C04B082F42
:107592000E94C40DDBCF8D010E949530E4E00C9473
:1075A2009F4E6AC00E940C0F1091F40C163018F016
:1075B20010E01093F40C2091F40C30E0F901EB5040
:1075C200F34F0083E4EFFCE010811395108305353F
:1075D20051F50091F40C0250073008F00A5F10E0F8
:1075E200F801EB50F34F00810F3FE9F400E0009304
:1075F200F40C0FEF2091F40C30E0F901EB50F34F53
:107602000083E4EFFCE000810395008305E520910F
:10761200F40C30E0F901EB50F34F0083E4EFFCE0AF
:107622000081039500830091F40C063029F5009146
:10763200F50C0F3F09F50091F60C0535E9F40091C0
:10764200F70C1091F80C10950117B1F40091F90C98
:107652001091FA0C1095011779F401E00093F30CE4
:107662003091F90C20E00091F70C10E0020F131F8B
:10767200EEEDFCE0008311830091FE0C1091FD0CF5
:10768200011709F08FCF08959A938A93C901083C94
:1076920009F0CFC0183151F4082F092B21F402E070
:1076A2000093DB0C01C18C0130DFFEC01A3111F0F6
:1076B2001B3149F5E0EEFCE0808391830FEF0E94DD
:1076C200DB0D05E50E94DB0DE0EEFCE0008111819F
:1076D2000E94DB0DE0EEFCE00081118100950E942A
:1076E200DB0DE0EEFCE000811181012F10E00E9431
:1076F200DB0DE0EEFCE000811181012F10E000952E
:107702000E94DB0DD1C01F3159F4882311F401E02E
:1077120001C000E0102F10FDAB9A10FFAB98C4C05F
:107722001232A1F540E050E010E020E030E000E04D
:107732000E94B10C002309F4B7C0E4EEFCE0008122
:1077420011810817190739F040E050E010E09C0160
:1077520001E00E94B10CE7E5F9E00381148108170A
:10776200190709F4A1C0E7E5F9E083839483082FA0
:1077720023E030E0A9010E94BE4D892F90E0082F3E
:1077820024E030E0A9010E94BE4D8EC0113229F4DE
:10779200E1EFFCE08083918387C0153221F48C01F4
:1077A2000E945C0E81C0163251F48C010E945C0E64
:1077B2000DE00E94DB0D0AE00E94DB0D75C018325D
:1077C200A1F540E050E010E020E030E000E00E944F
:1077D200B10C002309F468C0E6EEFCE000811181DF
:1077E2000817190739F0AC0110E020E030E004E09E
:1077F2000E94B10CE7E5F9E0018512850817190727
:1078020009F452C0E7E5F9E081879287082F29E061
:1078120030E0A9010E94BE4D892F90E0082F2AE096
:1078220030E0A9010E94BE4D3FC002E010E8D5D46D
:107832003BC00436F0F00D36E0F42091DD0C22233B
:1078420039F021E02093100D2091100D2223E1F751
:10785200EBE3F7E1212F30E0E20FF31F2491223016
:1078620021F49C010E94874D1FC0282F0E947F4D4A
:107872001BC02091DD0C222339F021E02093100D52
:107882002091100D2223E1F7E3E0F7E1212F30E010
:10789200E20FF31F2491223021F49C010E94874DB4
:1078A20003C0282F0E947F4D899199910895083C29
:1078B20009F0E4C0183181F4EAEEFCE000811181A4
:1078C200012B29F4ECEEFCE0008111810895EAEE2F
:1078D200FCE0008111810895193121F40091DD0C41
:1078E20010E008951A3111F01B3129F4E0EEFCE0AA
:1078F2000081118108951C3111F01D3149F451DECE
:1079020000E00093F30CEEEDFCE00081118108959C
:107912001E3129F446DE0091F30C10E008951F3168
:1079220041F405B30695069506950095017010E0A1
:1079320008951232B1F540E050E010E020E030E06E
:1079420000E00E94B10C002339F1E7E5F9E0038180
:107952001481E4EEFCE02081318102171307E1F08B
:10796200E4EEFCE000811181E7E5F9E00383148392
:10797200E4EEFCE00081118123E030E0A9010E94E5
:10798200BE4DE4EEFCE000811181012F10E024E005
:1079920030E0A9010E94BE4DE7E5F9E003811481C0
:1079A2000895143269F440E050E010E020E030E045
:1079B20000E00E94B10CE2EEFCE00081118108952A
:1079C2001032B9F400E0809902C0006111E00C9914
:1079D20002C0086011E00D9902C0046011E00E9926
:1079E20002C0026011E00F9902C0016011E010E0D4
:1079F2000895113229F4E1EFFCE00081118108952C
:107A02001832B1F540E050E010E020E030E000E054
:107A12000E94B10C002339F1E7E5F9E001851285F6
:107A2200E6EEFCE02081318102171307E1F0E6EE79
:107A3200FCE000811181E7E5F9E001871287E6EEBB
:107A4200FCE00081118129E030E0A9010E94BE4DD5
:107A5200E6EEFCE000811181012F10E02AE030E027
:107A6200A9010E94BE4DE7E5F9E00185128508955E
:107A720001E010E8B2D30FEF1FEF08950436E8F0EB
:107A82000E36D8F42091DD0C222339F021E0209328
:107A9200100D2091100D2223E1F7EBE3F7E1212FE6
:107AA20030E0E20FF31F2491223019F40E94694D55
:107AB20008950E945A4D10E008950F31D8F4209194
:107AC200DD0C222339F021E02093100D2091100DBE
:107AD2002223E1F7E3E0F7E1212F30E0E20FF31F89
:107AE2002491223019F40E94694D08950E945A4D42
:107AF20010E0089500E010E008959A938A93E1E17E
:107B0200FDE00081118198012F5F3F4FE1E1FDE02F
:107B12002083318320E030E0005010462F4F3F4F4A
:107B2200F801322F3BBF0690002D10E01BBFE1E1B0
:107B3200FDE0408151819A012F5F3F4FE1E1FDE07D
:107B42002083318360E070E0405050466F4F7F4F9A
:107B5200FA01362F3BBF0690202D10E01BBFE1E15A
:107B6200FDE040815181CA010196E1E1FDE080839F
:107B7200918360E070E0405050466F4F7F4FFA01B2
:107B8200362F3BBF069010E01BBF002321F4102DBF
:107B9200022F8DDE4EC0023061F4102D30E0220F34
:107BA200331FF901E35EF24F20813181022F7FDE24
:107BB20040C0013069F4002D10E0000F111FF801E0
:107BC200E35EF24F00811181102F022F70DE31C06F
:107BD2000330A9F4002D10E0000F111FF801E35E3D
:107BE200F24F00811181102F30E0220F331FF90173
:107BF200E35EF24F20813181022F59DE1AC0043038
:107C020039F4502D40E0022F10E0040F151F11C06F
:107C1200053069F4102D00E030E0200F311F220FF3
:107C2200331FF901E35EF24F0081118102C000E0CF
:107C320010E08991999108950E948E4EA801E1E188
:107C4200FDE00081118198012F5F3F4FE1E1FDE0EE
:107C52002083318320E030E0005010462F4F3F4F09
:107C6200F801322F3BBF0690002D10E01BBFE1E16F
:107C7200FDE000801180C0010196E1E1FDE080831A
:107C82009183C001A0E0B0E080509046AF4FBF4F5B
:107C9200FC013A2F3BBF0690602D10E01BBFE1E1D3
:107CA200FDE000801180C0010196E1E1FDE08083EA
:107CB2009183C001A0E0B0E080509046AF4FBF4F2B
:107CC200FC013A2F3BBF069010E01BBF002329F4B2
:107CD2009A01102D062FD8DC4BC0023069F49A01AC
:107CE200102D70E0660F771FFB01E35EF24F4081BB
:107CF2005181042FC9DC3CC0013071F49A01002D7E
:107D020010E0000F111FF801E35EF24F00811181B4
:107D1200102F062FB9DC2CC00330B1F49A01002DCC
:107D220010E0000F111FF801E35EF24F0081118194
:107D3200102F70E0660F771FFB01E35EF24F408168
:107D42005181042FA1DC14C0043021F407E010E0BB
:107D520044D20EC0053061F4102D00E070E0600FD7
:107D6200711F660F771FFB01E35EF24F4083518361
:107D7200E4E00C949F4EC1DEE3E1FDE00083118359
:107D8200E1E1FDE00081118198012F5F3F4FE1E1C8
:107D9200FDE02083318320E030E0005010462F4F79
:107DA2003F4FF801322F3BBF069000E00BBF00921D
:107DB200190DA3DEE5E1FDE0008311830091190DA9
:107DC200002379F4E3E1FDE000811181E5E1FDE0CA
:107DD200208131810217130711F401E0089500E0B8
:107DE20008950091190D013079F4E5E1FDE000817B
:107DF2001181E3E1FDE0208131810217130710F4C4
:107E020001E0089500E008950091190D023079F41F
:107E1200E3E1FDE000811181E5E1FDE020813181B6
:107E22000217130710F001E0089500E00895009191
:107E3200190D033079F4E3E1FDE000811181E5E100
:107E4200FDE0208131810217130710F401E008954B
:107E520000E008950091190D043079F4E5E1FDE0A8
:107E620000811181E3E1FDE02081318102171307D6
:107E720010F001E0089500E008950091190D053019
:107E820079F4E3E1FDE000811181E5E1FDE020818B
:107E920031810217130711F001E0089500E00895FF
:107EA20005E010E09AD100E0089500911A0D01302A
:107EB20061F400911C0D002331F000911B0D002391
:107EC20011F001E0089500E0089500911A0D0230CA
:107ED20061F400911C0D002321F400911B0D00237D
:107EE20011F001E0089500E0089506E010E075D178
:107EF20000E008959A938A930230C9F0E1E1FDE02F
:107F0200408151819A012F5F3F4FE1E1FDE02083E3
:107F1200318360E070E0405050466F4F7F4FFA016E
:107F2200362F3BBF069010E01BBF0092180D109138
:107F3200180D1F5F09F440C1125091F01A9509F112
:107F42001A9509F44CC01A9509F4F2C01A9509F46D
:107F5200FBC01A9509F407C11A9509F41CC137C16F
:107F6200002331F0CADDE1E1FDE00083118332C17B
:107F7200E1E1FDE0008111810D5F1F4F008311835C
:107F820029C1002319F1E1E1FDE0008111810D5FBA
:107F92001F4F00831183B1DDE5E1FDE00083118312
:107FA200E1E1FDE000811181065010400083118360
:107FB200E5E1FDE0008111813FDEE1E1FDE00081CC
:107FC20011810D5F1F4F0083118304C1E1E1FDE0C8
:107FD200008111810A5F1F4F00831183FBC00023C0
:107FE20009F49DC0E1E1FDE0008111810D5F1F4FA9
:107FF2000083118382DDE3E1FDE000831183E1E18F
:10800200FDE00081118198012F5F3F4FE1E1FDE02A
:108012002083318320E030E0005010462F4F3F4F45
:10802200F801322F3BBF069000E00BBF0092190D02
:1080320064DDE5E1FDE0008311830091190D002369
:1080420059F4E3E1FDE000811181E5E1FDE0808189
:108052009181800F911F50C00091190D013059F488
:10806200E3E1FDE080819181E5E1FDE000811181A4
:10807200801B910B41C00091190D023061F4E3E1C4
:10808200FDE000811181E5E1FDE0408151810E9426
:10809200D04DC80131C00091190D033061F4E3E104
:1080A200FDE000811181E5E1FDE0408151810E9406
:1080B200EC4DC80121C00091190D003159F4E3E1E2
:1080C200FDE000811181E5E1FDE080819181802365
:1080D200912312C00091190D013159F4E3E1FDE041
:1080E20000811181E5E1FDE080819181802B912B5E
:1080F20003C004E010E071D0E1E1FDE000811181F4
:108102000A501040008311838C0196DDE1E1FDE00D
:1081120000811181095F1F4F008311835BC0E1E180
:10812200FDE000811181065F1F4F0083118352C061
:10813200002309F04FC0E1E1FDE000811181E1E19E
:10814200FDE00083118346C0002321F00BE1009380
:10815200170D40C0E1E1FDE000811181E1E1FDE0A8
:108162000083118337C0002369F0E1E1FDE0008163
:1081720011810D5F1F4F61D2C0DCE1E1FDE00083A0
:10818200118328C0E1E1FDE0008111810D5F1F4FE5
:10819200008311831FC0002331F079D2E1E1FDE0B9
:1081A2000083118317C0E1E1FDE000811181E1E16B
:1081B200FDE0008311830EC0002361F4E1E1FDE0E4
:1081C20000811181E1E1FDE00083118303C003E13D
:1081D20010E003D08991999108959A938A93C801E6
:1081E200E7E6F9E0008101FF1AC00AE515E10E9405
:1081F200C04B8C010E94E20E0BE50E94DB0DE1E117
:10820200FDE0008111810E94E20E0AE30E94DB0D73
:108212000091180D0E94C40D0DE50E94DB0D89919D
:10822200999108950E948F4EA02FAA2311F4959838
:10823200969A00E010E0E1E1FDE00083118380E026
:1082420090E204E00093180DAA2321F00BE115E15E
:108252000E94C04B00E00093170D05C002E04ADE09
:10826200AA2309F013D10091170D0B3109F407C1AC
:10827200E1E1FDE020813181203000EC300708F09F
:10828200FEC00091180D053009F4F9C0E1E1FDE0EE
:10829200008111810817190708F0F1C0E1E1FDE042
:1082A2000081118198012F5F3F4FE1E1FDE02083C2
:1082B200318320E030E0005010462F4F3F4FF8014D
:1082C200322F3BBF069000E00BBF0092180DE8E191
:1082D200FDE0008107FFC2CF0091180D005849F060
:1082E2000A9509F46FC00A9509F4B0C00A95B1F174
:1082F200C2C041DD00931B0D00911B0D00931C0DAC
:10830200E1E1FDE00081118198012F5F3F4FE1E142
:10831200FDE02083318320E030E0005010462F4FF3
:108322003F4FF801322F3BBF069000E00BBF009297
:108332001A0DAA2309F0AAD000911A0D002309F000
:1083420092CF00911C0DD6DDAA2309F48CCF0091A7
:108352001C0D002309F487CF99D085CF0CDD009343
:108362001B0DA3DD00931C0DE1E1FDE000811181F5
:1083720098012F5F3F4FE1E1FDE02083318320E050
:1083820030E0005010462F4F3F4FF801322F3BBFD5
:10839200069000E00BBF00921A0DAA2309F076D0D6
:1083A20000911A0D002309F05ECF00911C0DA2DD91
:1083B200AA2309F458CF00911C0D002309F453CFCE
:1083C20065D051CF00911C0D002359F0E1E1FDE091
:1083D20000811181085F1F4F0083118300E08ADD55
:1083E20042CFC9DC00931B0D00911B0D00931C0DA5
:1083F200E1E1FDE00081118198012F5F3F4FE1E152
:10840200FDE02083318320E030E0005010462F4F02
:108412003F4FF801322F3BBF069000E00BBF0092A6
:108422001A0DAA2309F032D000911A0D002309F087
:108432001ACF00911C0D5EDDAA2309F414CF00911E
:108442001C0D002309F40FCF21D00DCFAA2309F070
:108452001DD000911C0D002311F401E001C000E0C9
:1084620049DDAA2309F4FFCE00911C0D002309F077
:10847200FACE0CD0F8CE00E110E0AFDEF4CE0091DF
:10848200DD0C0023E1F7E3E00C94A04E0CE810E0D1
:108492000E94C04B66D00DE20E94DB0D0091180DC8
:1084A2000E94C40D0AE30E94DB0D00E20E94DB0D74
:1084B20000911B0D0E94C40D0DE30E94DB0D08E22A
:1084C2000E94DB0DE3E1FDE0008111810E94E20EDA
:1084D2000CE20E94DB0D00E20E94DB0D0091190DFF
:1084E2000E94C40D0CE20E94DB0D00E20E94DB0D33
:1084F200E5E1FDE0008111810E94E20E09E20E94A5
:10850200DB0D00E20E94DB0D00911A0D0E94C40DEA
:108512000BE70E94DB0D00911C0D0E94C40D0DE7BC
:108522000E94DB0D0BE50E94DB0DE1E1FDE0008125
:1085320011810E94E20E0DE50E94DB0D0E940C0FDC
:108542000093170D0091170D0B3151F40DE415E155
:108552000E94C04BE1E1FDE0008111810E94E20E28
:1085620008950091180D003829F404E615E10E94DF
:10857200C04B08950091180D013829F40CE615E15D
:108582000E94C04B08950091180D023829F404E7A7
:1085920015E10E94C04B08950091180D033829F48B
:1085A2000CE715E10E94C04B08950091180D0130AF
:1085B20029F404E815E10E94C04B08950091180DBA
:1085C200023029F40CE815E10E94C04B0895009195
:1085D200180D033029F404E915E10E94C04B0895F7
:1085E2000091180D043029F40CE915E10E94C04BEA
:1085F20008950091180D053029F404EA15E10E944E
:10860200C04B08950091180D063029F40CEA15E1CB
:108612000E94C04B08950091180D073029F404EB15
:1086220015E10E94C04B08950091180D0F3F21F4EF
:108632000CEB15E10E94C04B08952091AB0D2A303E
:1086420010F52091AB0D30E0220F331FF901EF57E7
:10865200F24F00831183EBEAFDE000810395008372
:1086620020911C0D30E00091AB0D10E0000F111FA6
:10867200F801EF57F24F20833183EBEAFDE00081EE
:1086820003950083089509E010E0A7DD08950091A5
:10869200AB0D0023E9F0EBEAFDE000810A950083CF
:1086A20010E0000F111FF801EF57F24F0081118106
:1086B20000931C0DEBEAFDE000810A95008310E0B7
:1086C200000F111FF801EF57F24F00811181089539
:1086D2000AE010E082DD0FEF1FEF08950E948E4E38
:1086E20000916110002309F0D3C000915E090130AE
:1086F20009F094C0E4EDFDE002811381012B09F43D
:108702005AC000E00093CB0D00E010E0E0EDFDE088
:108712000083118300E010E0E2E6F0E100831183C0
:1087220001E000936110E4EDFDE00081118145E07C
:1087320050E00E94EC4D10E0ECECFDE00083118370
:10874200ECECFDE080819181E4EDFDE0028113819A
:1087520045E050E00E94EC4D10E0801B910BEEECE6
:10876200FDE080839183EEECFDE0208131812437AE
:1087720000E0300720F003E00093DD0D27C2EEECAD
:10878200FDE020813181223700E0300720F007E050
:108792000093DD0D1BC2EEECFDE02081318120371C
:1087A20000E0300720F00FE00093DD0D0FC20FE074
:1087B2000093DD0D0BC20091CB0D0370002309F075
:1087C20005C2E4EDFDE00081118145E050E00E9428
:1087D200EC4D10E0ECECFDE000831183ECECFDE0ED
:1087E20080819181E4EDFDE00281138145E050E05A
:1087F2000E94EC4D10E0801B910BEEECFDE08083BB
:108802009183EEECFDE020813181293500E03007D3
:1088120008F0DCC10FE70093DD0DD8C1E4EDFDE007
:1088220002811381012B09F0D1C10091CB0D03709C
:10883200002309F0CBC1E4EDFDE00081118145E0A8
:1088420050E00E94EC4D10E0ECECFDE0008311835F
:10885200ECECFDE080819181E4EDFDE00281138189
:1088620045E050E00E94EC4D10E0801B910BEEECD5
:10887200FDE080839183EEECFDE02081318129359A
:1088820000E0300708F0A2C10FE70093DD0D9EC1A2
:1088920000916110013009F04AC1E4EDFDE002816E
:1088A2001381012B61F400E010E01BBD0ABD00E062
:1088B2000093DD0DA89800E00093611087C100913C
:1088C200CB0D0F71002329F400E010E01BBD0ABD9F
:1088D2007DC10091CB0D0F71023009F077C1E4ED3B
:1088E200FDE00081118145E050E00E94EC4D10E076
:1088F200ECECFDE000831183ECECFDE080819181E2
:10890200E4EDFDE00281138145E050E00E94EC4D70
:1089120010E0801B910BEEECFDE080839183E0ED93
:10892200FDE000811181EEECFDE020813181021732
:10893200130740F4EEECFDE000811181E0EDFDE073
:1089420000831183E3E0F6E1A8EDBDE00D911C91F7
:1089520011971695079516950795E00FF11F04914B
:1089620010E0E2EDFDE000831183EEECFDE000811A
:1089720011810A5F1F4FECECFDE02081318102176B
:10898200130718F00FEF13E010C00AEF17E1ECEC39
:10899200FDE040815181EEECFDE020813181421BFE
:1089A200530B465050400E94EC4D003024E0120719
:1089B20010F00FEF13E01BBD0ABDA2EDBDE0ED917B
:1089C200FC911197F69720F003E00093DD0D32C081
:1089D200A2EDBDE0ED91FC911197F49720F007E034
:1089E2000093DD0D27C0EEECFDE0208131812437BC
:1089F20000E0300720F003E00093DD0D1BC0EEEC39
:108A0200FDE020813181223700E0300720F007E0CD
:108A12000093DD0D0FC0EEECFDE0208131812037A7
:108A220000E0300720F00FE00093DD0D03C00FE0FF
:108A32000093DD0DE2E6F0E1008111810F5F1F4F2F
:108A420000831183E2E6F0E120813181283601E0E2
:108A5200300758F000E010E01BBD0ABD0FEF009395
:108A6200DD0D02E800936110B1C0EEECFDE0208163
:108A72003181263700E0300758F000E010E01BBDDE
:108A82000ABD0FEF0093DD0D01E8009361109EC057
:108A9200E0EDFDE0008111810C531040EEECFDE0B1
:108AA200208131810217130798F0EEECFDE020815E
:108AB2003181253600E0300758F000E010E01BBDA0
:108AC2000ABD0FEF0093DD0D03E8009361107EC035
:108AD200E2EDFDE0208131812C3300E0300758F0D7
:108AE20000E010E01BBD0ABD0FEF0093DD0D04E8AE
:108AF200009361106BC0A2EDBDE0ED91FC91119766
:108B0200F89708F463C0EEECFDE020813181203754
:108B120000E0300708F45AC000E010E01BBD0ABDB7
:108B22000FEF0093DD0D04E8009361104FC0009138
:108B32005E09023041F002E000935E0927E030E076
:108B4200A9010E94BE4DE4EDFDE002811381012BDB
:108B5200C1F400E010E01BBD0ABD00E00093DD0D92
:108B6200A89800E00093611000915E09002371F162
:108B720000E000935E0927E030E0A9010E94BE4DAB
:108B820025C00091CB0D0F71002301F5E4EDFDE04E
:108B92000081118145E050E00E94EC4D10E0ECECC8
:108BA200FDE000831183ECECFDE080819181E4ED36
:108BB200FDE00281138145E050E00E94EC4D10E09F
:108BC200801B910BEEECFDE080839183E4E00C943A
:108BD2009F4E07EE06B900E010E01BBD0ABD03EC94
:108BE2000FBD02E00EBD03E00093DC0DECEDFDE0F5
:108BF200008103950083037007B901E010E00E9431
:108C02005C0C24B135B10091DC0D10E003701070E2
:108C1200000F111FF801EC52F24F20833183ECED6B
:108C2200FDE0008103950083037007B901E010E0C5
:108C32000E945C0C24B135B10091DC0D10E0037090
:108C42001070000F111FF801EC52F24F2083318394
:108C5200ECEDFDE0008103950083037007B901E0AC
:108C620010E00E945C0C24B135B10091DC0D10E0E3
:108C720003701070000F111FF801EC52F24F2083A5
:108C82003183ECEDFDE0008103950083037007B9A9
:108C920001E010E00E945C0C24B135B10091DC0DC2
:108CA20010E003701070000F111FF801EC52F24F28
:108CB2002083318308950E948F4E1A981B9A0E9436
:108CC200D80BA89800E0009365090093660900E0BC
:108CD200009367090093680900E00093DD0C00E04F
:108CE2000093EE0C22E030E0A9010E94B24D0F3F4A
:108CF200A9F021E030E0A9010E94B24D0F3F71F0CE
:108D020023EF3FE0A9010E94B24D033038F427E07F
:108D120030E0A9010E94B24D033048F101E0009316
:108D2200580921E030E0A9010E94BE4D02E2009301
:108D3200570920E030E0A9010E94BE4D00E022E088
:108D420030E0A9010E94BE4D80E023EF3FE0082FF2
:108D5200A9010E94BE4D0AE00093EE0C00E00093D0
:108D62005E0927E030E0A9010E94BE4D37C021E034
:108D720030E0A9010E94B24D0093580920E030E092
:108D8200A9010E94B24D0093570923EF3FE0A901C8
:108D92000E94B24D802F23E030E0A9010E94B24D23
:108DA20000935A0924E030E0A9010E94B24D0093D9
:108DB2005B0929E030E0A9010E94B24D00936009ED
:108DC2002AE030E0A9010E94B24D0093610927E038
:108DD20030E0A9010E94B24D00935E0900E00093C9
:108DE2005F0911E020E830E000E00E94B90B21E0C9
:108DF2001091570900E00E94280C21E012E201E0E4
:108E02000E94280C00E00093650900936609E1DEE8
:108E1200789424EF3FE0A9010E94B24D053519F480
:108E220000E0C8D45EC1833038F080E023EF3FE039
:108E3200082FA9010E94BE4D94B700E004BF21EFA4
:108E42003FE0A9010E94B24D002361F0923051F43B
:108E52008395833008F080E023EF3FE0082FA901DB
:108E62000E94BE4D9A70992361F400915E0900231D
:108E720041F000E000935E0927E030E0A9010E9482
:108E8200BE4D21EF3FE0A9010E94B24D013031F009
:108E920001E021EF3FE0A9010E94BE4D00915E0971
:108EA200023009F05DC000E8009361100FEF0093FB
:108EB200DD0D56C090E0809B04C002E310E00E94EA
:108EC2005C0C0091FE0C1091FD0C011769F00E94E0
:108ED2000C0FA02FA53521F40091FD0C0093FE0C80
:108EE200082F0E94DB0D01C0A0E0882311F4AC988A
:108EF20007C0813011F4AD9803C0823009F4AE98F6
:108F0200933209F046C0A33209F043C004E110E0F5
:108F12000E945C0C08E001BD809B04C002E310E0EB
:108F22000E945C0C0C991CC002E310E00E945C0CD5
:108F320000915E09002371F4E4EDFDE002811381EA
:108F4200012B41F001E000935E0927E030E0A90126
:108F52000E94BE4D0C9BFECF02E310E00E945C0C0F
:108F6200809B31C0AD9AAC9AAE9A0091FE0C1091E2
:108F7200FD0C011709F49ECF0E940C0F902F95351E
:108F820021F40091FD0C0093FE0C082F0E94DB0DD2
:108F920092CF993011F0A93089F404E110E00E94D7
:108FA2005C0C08E001BD8395833008F080E023EF7C
:108FB2003FE0082FA9010E94BE4DAECF9D3019F0AF
:108FC200AD3009F0A9CF21EF3FE0A9010E94B24DD7
:108FD200002331F000E021EF3FE0A9010E94BE4DE5
:108FE200809BFECF04E110E00E945C0C00E910E0DF
:108FF200C6D38ED3882391F401E0DCD3902F0CE802
:1090020010E0BDD3092F0E94200F08E512E0B7D36C
:1090120001E0009367090E94300FFDCF00915709CC
:10902200013059F101E0009357092091570914E0EA
:109032000EEF64D505E912E0A2D300E814E82EE1B0
:1090420030E04091570950E060E070E04F5F5F4FC1
:109052006F4F7F4F0E945B4E0E94030E00EB12E0A7
:109062008ED30091570920E030E0A9010E94BE4D45
:1090720009B904EF11E00E945C0C01E010E0E8ED98
:10908200FCE00083118301E095D3902F0CE810E0FF
:1090920076D3092F0E94200F08E512E070D307E073
:1090A200009367090E94CA21E4EDFDE0208131812D
:1090B200273302E0300730F023E333E012E20EEF11
:1090C20025D505C02FEF33E012E20EEF1FD5813018
:1090D20071F401E010E0E8EDFCE0008311830E94EE
:1090E200E72203E0009367090E945B2416C08230E6
:1090F200A1F404E610E00E945C0C02E00093670910
:1091020000E00E94134104E610E00E945C0C04E1BE
:1091120010E00E945C0C08E001BDFFCFFA93EA93D5
:109122004A933A932A931A930A933FB74BB700E0B4
:109132000BBFAA9820919C000091FD0C10E00F70CB
:109142001070F801E150F34F2083EDEFFCE0008155
:10915200039500834BBF3FBF099119912991399122
:109162004991E991F9911895FA93EA934A933A93BE
:109172002A931A930A933FB74BB700E00BBF0091B3
:109182006509102F1395109365092CB110E0F801B1
:10919200EB56F94F20834BBF3FBF0991199129919B
:1091A20039914991E991F99118952497AA98A9982A
:1091B20008EA10E0E4D223C00E940C0F0E94D70DEF
:1091C2005E9A0091FE0C1091FD0C0117A9F75E9BAF
:1091D200FECF1A981B9A0091660910916509011732
:1091E20071F00091660910E0F801EB56F94F008129
:1091F200E6E6F9E01081139510830E94DB0D0091E1
:10920200FE0C1091FD0C011731F31B981A9AD9CF5D
:109212000E948B4EAA98A99808EA10E0B0D218C012
:109222005E9BFECF1A981B9A009166091091650900
:10923200011771F00091660910E0F801EB56F94F41
:109242000081E6E6F9E01081139510830E94DB0DA0
:109252000091FE0C1091FD0C011731F31B981A9A24
:109262001CC0FC013A2F3BBF0690002D10E01BBF33
:109272008F5F9F4FAF4FBF4F600E0E94D70D5E9A18
:1092820001E0400E00E0501E0FEF401607E15006CD
:1092920040F3062D0E94D70D5E9A0091FE0C1091AC
:1092A200FD0C011709F4BCCF0E940C0F0E3741F4DC
:1092B20080E090ECA0E0B0E0662444245524E4CFA2
:1092C2000E94D70D5E9AE9CF0E948D4E902F4424C2
:1092D2009F3F29F400E014EF21E030E004C008EEE3
:1092E20013E020E030E080E013C04091660950E0D6
:1092F200FA01EB56F94F4081E6E6F9E050815395C9
:109302005083682F70E0FB01E95EF74F408383953D
:109312008917D8F440E050E060E070E00090660900
:1093220010906509011479F40A011B01A001B10131
:109332004F5F5F4F6F4F7F4F0015110522053305B9
:1093420068F744244394442081F2A82FB0E00091AE
:10935200CD080E3F09F470C0442071F09F3F61F0C8
:10936200E7E6F9E0008100FF03C00FE11DE007D24C
:109372000091650900936609A43008F45DC000916C
:1093820017080F3F21F4009118080F3F71F0E7E62C
:10939200F9E0008100FF03C004E31DE0F0D1009179
:1093A20065090093660900E048C000911908109110
:1093B200CD08011771F0E7E6F9E0008100FF03C074
:1093C2000AE41DE0DCD1009165090093660900E022
:1093D20034C020911A0830E00A2F10E004501040E7
:1093E2002017310771F0E7E6F9E0008100FF03C0C2
:1093F20000E61DE0C4D1009165090093660900E012
:109402001CC082E007C090E0FC01E95EF74F0081DA
:10941200B00F83958A17B8F3BF3F71F0E7E6F9E022
:10942200008100FF03C006E71DE0A9D10091650994
:109432000093660900E001C00A2FE5E00C949E4EFD
:109442000E948E4E3FEF3093CB083FEF3093CC0813
:109452000093CD08022F0E5F0093CE081093CF0821
:1094620080E00DC090E0FC01EB56F84F0081A82F80
:10947200B0E01596FD01E553F74F008383958217FF
:1094820088F300E02A5FA22F82E007C090E0FC018F
:10949200E553F74F1081010F839590E0EA2FF0E03A
:1094A20031978E179F0794F3009590E0FC01E553E6
:1094B200F74F00831B981A9A80E009C05E9A90E0E9
:1094C200FC01E553F74F00810E94D70D83958A175F
:1094D200A8F35E9BFECF1A981B9A0A2FE4E00C9425
:1094E2009F4E0E948E4ED801922F992359F40091DB
:1094F200CD080E3F21F400EF11E041D103C001E19C
:1095020012E03DD180E00CC0082F10E0FD01E00F19
:10951200F11F00810E94930E00E20E94DB0D8395F1
:10952200891790F301E412E02AD1092F0E94200F3B
:10953200E4E00C949F4E0E948C4E802F912F422E7D
:1095420001E00093DC0CB0E02DC040E050E060E0B0
:1095520070E0F0E08A019B01A801B9014F5F5F4F03
:109562006F4F7F4F083EE3E01E07E0E02E07E0E08A
:109572003E0798F40091660910916509011751F3AD
:10958200009165090093660940E050E060E070E0F8
:109592000F2FF02FF3950536E8F20091650900933D
:1095A2006609B395B23008F051C000916509009385
:1095B2006609242D192F082F43DFA02F913061F463
:1095C2008E3F29F455245A945092690930C006E01E
:1095D200502E509269092BC0923039F45090960760
:1095E20006E0500E5092690922C08E3FC1F08F31C1
:1095F20040F4082F10E0F801E659F64F00810238D6
:1096020070F0843680F08E3670F4082F10E0045625
:109612001040F801E657F64F0081023820F4552435
:109622005092690913C006E0502E509269095520E4
:1096320009F4B7CF052D48DE009369090091690945
:10964200051521F00FEF501609F07FCF00E00093CF
:10965200DC0C00916909051509F443C00091CD089D
:109662000E3FF9F1E7E6F9E0008100FF15C00DEDCC
:109672001DE085D0082F0E94200F07EB10E07FD05D
:109682002A2F0BEC18E02DDF09EC10E078D02091A6
:10969200690907E118E025DFE7E6F9E0008101FF4B
:1096A2001EC000E011E80E94EE40082F0E94930EB7
:1096B20000E20E94DB0D092F0E94930E00E20E943D
:1096C200DB0D009195070E94930E00E20E94DB0DD4
:1096D200009196070E94930E00E20E94DB0D00E0CB
:1096E20014C000916809002379F007EB10E047D01D
:1096F2002A2F0BEC18E0F5DE09EC10E040D02091A7
:10970200690907E118E0EDDE01E0E6E00C949D4E08
:109712000BED10E034D000E814E82EE130E0409187
:10972200990050E060E070E04F5F5F4F6F4F7F4FF6
:109732000E945B4E0E94030E00E20E94DB0D00EBD2
:1097420012E01DD00CE20E94DB0D05EE10E017D0F6
:1097520000E814E82EE130E049B150E060E070E04A
:109762004F5F5F4F6F4F7F4F0E945B4E0E94030E11
:1097720000E20E94DB0D00EB12E001D00895EF97AA
:10978200EF97A49720E001C02395203A60F430E0DF
:10979200F801E20FF31F4491FE0130E0E20FF31FE4
:1097A2004083442389F78E010E94FF0EEF96EF96C5
:1097B200A49608950E948E4EB02FBB2361F00CE850
:1097C20010E0DDDF09E40E94DB0D04E40E94DB0D02
:1097D2000AE30E94DB0D90E020E011E00EEFABDE29
:1097E20000916909002309F494C0A0E00EC08436F8
:1097F20058F08E3648F420E0082F10E0045610404E
:10980200F801E657F64F2083A39500916909A01746
:1098120008F07FC00A2F10E0F801E95EF74F0081DF
:109822000F3F91F70A2F10E00F5F1F4FF801E95E1B
:10983200F74F00810F3F41F70A2F10E00E5F1F4FD5
:10984200F801E95EF74F80810A2F10E00D5F1F4F8C
:10985200F801E95EF74F0081023009F04FC00A2F8C
:1098620010E00E5F1F4FF801E95EF74F208130E0F4
:109872000A2F10E00D5F1F4FF801E95EF74F40819C
:1098820050E0420F531F0A2F10E00C5F1F4FF801E8
:10989200E95EF74F208130E0240F351F0A2F10E0D8
:1098A2000B5F1F4FF801E95EF74F008110E0020FD6
:1098B200131F0F3F20E0120709F58F3140F420E813
:1098C200082F10E0F801E659F64F20830DC08436C8
:1098D20058F08E3648F420E8082F10E00456104065
:1098E200F801E657F64F2083BB2331F0082F0E9480
:1098F200930E00E20E94DB0D939586CF8F3108F024
:1099020076CF20E0082F10E0F801E659F64F2083C9
:109912007BCF40EC50EE60E070E080E059C002E0A6
:10992200809F8001212F220F220B322F040F151F3F
:10993200261F371F0F5F1F4F2F4F3F4FF801322F48
:109942003BBF0690102D00E00BBF00E022E0829F9B
:10995200212C220C2208322C040E151E261E371E24
:10996200F001322D3BBF069020E02BBF1124000EE8
:10997200111E082F10E0000F111FF801EB56F64FD1
:1099820000821182082F10E0000F111FF801EB5620
:10999200F64F20813181203000E4300769F0082F32
:1099A20010E0000F111FF801EB56F64F20813181B4
:1099B200203000E4300759F400E010E0282F30E0B6
:1099C200220F331FF901EB56F64F00831183839563
:1099D2008F3108F4A4CF80E012C014E2082F0E9455
:1099E200592F0060106222E0829F20E0020E22E0E6
:1099F200121EF001EB52F64F0083118383958F31D3
:109A020080F5082F10E0F801E659F64F0081002397
:109A1200A9F310E1082F4DD00068282F30E0F9019A
:109A2200E659F64F008315E0082F43D0002321F0BA
:109A320020E015E0082F62D018E1082F3AD001305B
:109A420061F61EE1082F0E94592F22E0829F20E03A
:109A5200020E22E0121EF001EB52F64F0083118338
:109A6200CDCF84E620C0A82FB0E0A456B040FD01BF
:109A7200E657F64F00810023A9F010E1082F19D014
:109A82000068A82FB0E0A456B040FD01E657F64F9B
:109A9200008315E0082F0DD0002321F020E015E00F
:109AA200082F2CD083958E36F0F2092FE4E00C9427
:109AB2009F4E1093950711E01093960722E012E053
:109AC2003ADD002319F000911C0808950FEF089564
:109AD2001093950712E01093960722E012E02BDD17
:109AE200002349F030911D0820E000911C0810E08D
:109AF200020F131F08950FEF1FEF0895109395079C
:109B02002093960722E013E016DD0895109395073F
:109B1200122F10939607232F30E02093970723E00C
:109B220013E009DD08950FE30DBF05E00EBFC0E0AD
:109B3200D5E00E94AA4E002311F00E94BC4E00E024
:109B42000BBF0E945C460E94DF4E0C94DF4EE199EF
:109B5200FECF08954F5F5F4FFADF4EBB5FBBE09AC7
:109B62000895FADF0DB308954F5F5F4F4EBB5FBBA1
:109B7200F894E29AE19A0FBE08950FB6E8DF0DBBA2
:109B8200F5CF0024E8E0EA9532F0001F001C04162D
:109B9200D0F3041AF8CF001F402D00950895002439
:109BA20011240030010741F01695079510F4040EB8
:109BB200151E440F551FF5CF002D112D08954A95FE
:109BC2001AF0000F111FFBCF08954A951AF016954F
:109BD2000795FBCF089500241124EFE0001F111F09
:109BE200001C111C0416150610F0041A150AEA9539
:109BF200AAF7001F111F402D512D009510950895B1
:109C020030952095109501951F4F2F4F3F4F089586
:109C120070956095509541955F4F6F4F7F4F0895B6
:109C22000024112422243324E02FE12BE22BE32B06
:109C320071F0369527951795079520F4040E151E99
:109C4200261E371E440F551F661F771FEDCF002DAE
:109C5200112D222D332D08954A952AF0000F111F40
:109C6200221F331FF9CF0895002411242224332404
:109C7200E0E2EA9592F0001F111F221F331F001C21
:109C8200111C221C331C041615062606370688F3FF
:109C9200041A150A260A370AECCF001F111F221FC9
:109CA200331F402D512D622D732D00951095209557
:109CB20030950895FF2777231AF4F1600E94094E28
:109CC20033231AF4F0950E94014E0E94354EF69508
:109CD20010F40E94014EF69510F40C94094E08956A
:109CE200AF93BF93B12FA02F3BBFD895EF5FFF4F2C
:109CF2003F4F0D9241505040B9F74BBFBF91AF91CA
:109D02000895FA92EA92DA92CA92BA92AA929A9230
:109D12008A927A926A925A924A92BA93AA939A939E
:109D22008A930895FF84EE84DD84CC84BB84AA8464
:109D3200998488847F806E805D804C80BB81AA81FB
:109D420099818881F0E00FB6F894CE0FDF1F0FBE25
:109D5200089501E0089520E002D0E9F708952D93D7
:109D620001501040202F212B08953BBF27913BB774
:109D7200F6DFD9F708950FE01EE92801F20130E07D
:109D82003BBF07911691F2013296A791B691F2016B
:109D92003496479157916691242F252B262B21F03B
:109DA200FA01362FE2DF01C0D6DF07E0400E00E005
:109DB200501EA2014D315E4908F3089500008895B6
:109DC200FECF141A1F24292E33383D4D151B202592
:109DD2002A2F343908080809090909090909090952
:109DE20009090909090909090808080808080808E9
:109DF200080808070700FF03020504070609080B05
:109E02000A0D0C0F0E111013121514FF005501400C
:109E1200051D9E00CF09950600000044554D5000D7
:109E220049440050494E47004700474F00445245BD
:109E3200534554005245534554005359535F5752AA
:109E42000041435400414354494F4E005245475F3D
:109E52005752005700575200575249544500535920
:109E62004E435F5752005357520043414C550044F2
:109E72004543004845580043414C430043414C444C
:109E8200000D0A205B4349443A005D2000524554CC
:109E92000052455455524E0052554E0048454C50C2
:109EA200004C004C544F5353005400544F53530032
:109EB20043494400544553540043484B0044454DE4
:109EC2004F004D4F4E49544F5200424155440053AA
:109ED2004541524348004C4544005343414E0055CE
:109EE2005044415445004400535445500042414CB3
:109EF200414E4345004F4646004F4E004E414D45B0
:109F020000434F5059005000504147450042004223
:109F120045464F5245004E004E45585400474F5457
:109F22004F004D4F4E0052450052005244005245E0
:109F3200414400480045584954005341560053419A
:109F42005645004E4557004D004D4952524F520062
:109F520053455400504C4159004900494E53455213
:109F6200540044454C455445004D4F56450053005E
:00000001FF
